:100000000C94CE020C94F6020C94F6020C94F602B8
:100010000C94F6020C94F6020C94F6020C94F60280
:100020000C94F6020C94F6020C94F6020C94F60270
:100030000C94F6020C94F6020C94F6020C94F60260
:100040000C944D2E0C94F6020C944A300C9498307B
:100050000C94F6020C94F6020C94F6020C94F60240
:100060000C94F6020C94F602BC1A961A591C351B15
:100070001F1B061CA81A591CD81A8D1A9F1AF51B8B
:10008000221BF71A421CB11AD31A741A491CE11B1D
:10009000EA1BFD1BF81B591C8C0390039503990365
:1000A000A303A803AF03B403BA03BF03C403C90384
:1000B000D003D803E003E603EB03F103FD030504DB
:1000C0000A04110418042004485454502F312E30CF
:1000D0002034303120556E617574686F72697A65AD
:1000E000640A436F6E74656E742D547970653A209E
:1000F000746578742F68746D6C0A3C68313E3430D6
:100100003120556E617574686F72697A65643C2F31
:1001100068313E0057616B652075700A004D61695A
:100120006E74656E616E63650A00206D730A004D22
:100130006F64652045434F200046696E2064656CFE
:100140006573746167650A004D6F64652064656C52
:100150006573746167650A00537263206164647239
:10016000657373203A20004C6E646B205472616397
:1001700065722076302E38642C202863294C652047
:100180004E6574206475204B65726D657572203202
:100190003031350A002C20476174657761793A2047
:1001A000002C204E65746D61736B3A20004950201D
:1001B000616464726573733A2000206D560A0020F2
:1001C0006D562C2056696E3A200020627974657352
:1001D0002C205663633A200046726565206D656D7C
:1001E0006F72793A20006261636B20746F2031393D
:1001F000322E3136382E312E32350A00646F6E655C
:100200000A0052657175657374696E6720495020E4
:1002100041646472657373202E2E2E20004661693E
:100220006C656420746F2061636365737320454E51
:100230004332384A36300A00454E4332384A363067
:100240002076657273696F6E2000646F6E650A00B8
:10025000496E697420454E4332384A3630202E2E7E
:100260002E004D6F64652064656275670A00436FF8
:100270006D6D616E64203A20003C68313E32303052
:10028000204F4B3C2F68313E00556E617574686F8E
:1002900072697A6564206163636573730A005365EC
:1002A000742054696D6520004D6F64652045434F8F
:1002B000206465736163746976650A004D616E71CF
:1002C000756520706172616D65747265730A0020D6
:1002D000636172616374657265730A005265637568
:1002E00020000A3C2F626F64793E0A3C2F68746DCF
:1002F0006C3E0A003C68746D6C3E3C686561643E0F
:100300003C7469746C653E4C6E646B20547261631E
:1003100065723C2F7469746C653E3C2F686561643E
:100320003E0A003C626F64793E3C68313E4C6E642C
:100330006B205472616365722076657273696F6EAB
:100340002076302E38643C2F68313E0A00485454E1
:10035000502F312E3020323030204F4B0D0A436F5A
:100360006E74656E742D547970653A207465787476
:100370002F68746D6C0D0A507261676D613A206E62
:100380006F2D63616368650D0A0D0A0041434300E8
:100390004144445200434D440044454C455354416C
:1003A00047450044554D5000454550524F4D00477C
:1003B00041544500484953544F004C4F4144004D6F
:1003C000414341004D41534B004D454D4F52590063
:1003D0004D455355524553004D4F444545434F00FD
:1003E000504152414D00504F5254005245534554D4
:1003F0000053455249414C444542554700535441EE
:100400004E4442590054494D4500555054494D45BC
:100410000056494E4D415800564F4C5441474500F7
:100420005741544348444F47000001080006040068
:10043000014500008200004000200D0A436F6E74E9
:10044000656E742D547970653A206170706C6963C3
:100450006174696F6E2F782D7777772D666F726D67
:100460002D75726C656E636F6465640D0A0D0A000C
:10047000436F6E74656E742D4C656E6774683A20B8
:10048000000D0A557365722D4167656E743A2045FB
:1004900074686572536869656C642F312E360D0A75
:1004A0004163636570743A202A2F2A0D0A436F6EE8
:1004B0006E656374696F6E3A20636C6F73650D0AC5
:1004C000000D0A0020485454502F312E310D0A4897
:1004D0006F73743A2000504F5354200020000D0ACF
:1004E000557365722D4167656E743A204574686571
:1004F00072536869656C642F312E360D0A4163634F
:100500006570743A20746578742F68746D6C0D0A88
:10051000436F6E6E656374696F6E3A20636C6F73C0
:10052000650D0A0D0A0020485454502F312E310D0C
:100530000A486F73743A20004745542000000000B9
:1005400000240027002A0000000000250028002BBE
:100550000000000000230026002900040404040415
:100560000404040202020202020303030303030160
:100570000204081020408001020408102001020437
:10058000081020000000070002010000030406001C
:100590000000000000000000FE06063211241FBE0D
:1005A000CFEFD8E0DEBFCDBF15E0A0E0B1E0ECE2D8
:1005B000FAE602C005900D92A63AB107D9F717E006
:1005C000A6EAB5E001C01D92A03FB107E1F715E032
:1005D000CCE9D5E004C02297FE010E94D934C83985
:1005E000D107C9F70E945C320C9414350C940000BA
:1005F000A0E0B0E0EEEFF2E00C94E534EC01A8806E
:10060000B980CA80DB80A114B104C104D10441F4D3
:1006100084E2A82E89EDB82E8BE5C82E87E0D82E6F
:10062000C601B5012DE133EF41E050E00E94BC343A
:1006300027EA31E440E050E00E9454347B018C0111
:10064000C601B5012DE133EF41E050E00E94BC341A
:10065000CA01B9012CEE34EF4FEF5FEF0E94543422
:100660006E0D7F1D801F911F97FF04C06150704069
:1006700080409048688379838A839B839B013F777E
:10068000C901CDB7DEB7EAE00C9401350E94F8024B
:1006900008958BE291E00E94F8020895A0E0B0E096
:1006A00080932B0190932C01A0932D01B0932E01E8
:1006B0000895FC0105900020E9F7809590958E0F34
:1006C0009F1F0895FB01DC014150504030F08D9197
:1006D0000590801919F40020B9F7881B990B08952B
:1006E000DC0101C06D9341505040E0F70895FB01DB
:1006F000DC014150504030F08D910190801919F487
:100700000020B9F7881B990B0895EF92FF920F9381
:100710001F93CF93DF93EC01A0E0B0E0EE24FF2421
:10072000870109C0F901EA0FFB1F8081E80EF11C67
:10073000011D111D1196A617B707A4F3452B69F0EB
:100740009B01442737FD4095542FB701C8010E94F3
:100750009A34C901DA017C018D01D801C701807F7B
:100760009070A070B07024E0B695A7959795879586
:100770002A95D1F78A3010F0895C01C0805DFE01B6
:10078000E258FB4F80839E012F5F3F4F6E2D6F70AD
:100790006A3010F0695C01C0605DF901E258FB4FFE
:1007A00060832F5F3F4FF901E258FB4F80E2808367
:1007B0002F5F3F4FC901DF91CF911F910F91FF90A4
:1007C000EF900895EF92FF920F931F93CF93DF93D3
:1007D000EC01FA0120E030E0EE24FF2487010AC09A
:1007E00081919191A0E0B0E0E80EF91E0A1F1B1F55
:1007F0002F5F3F4F261737079CF39B01442737FD98
:100800004095542FC801B7010E949A3479018A019A
:10081000D801C7016CE0B695A795979587956A951D
:10082000D1F78F708A3010F0895C01C0805DFE01C5
:10083000E258FB4F80839E012F5F3F4FBB27A12FC4
:10084000902F8F2D8F708A3010F0895C01C0805DF1
:10085000F901E258FB4F80832F5F3F4FD801C7015A
:10086000807F9070A070B07044E0B695A795979582
:1008700087954A95D1F78A3010F0895C01C0805D78
:10088000F901E258FB4F80832F5F3F4F4E2D4F7091
:100890004A3010F0495C01C0405DF901E258FB4F5D
:1008A00040832F5F3F4FF901E258FB4F80E2808386
:1008B0002F5F3F4FC901DF91CF911F910F91FF90A3
:1008C000EF9008959C01DB01CA01FCE1B695A79564
:1008D00097958795FA95D1F78A30910514F0895C40
:1008E00001C0805DF901E258FB4F80832F5F3F4FCD
:1008F000DB01CA0180709070A070BF708B2F9927A8
:10090000AA27BB278A30910514F0895C01C0805D5D
:10091000F901E258FB4F80832F5F3F4FDB01CA0193
:1009200080709070A07FB070F4E1B695A795979510
:100930008795FA95D1F78A30910514F0895C01C04A
:10094000805DF901E258FB4F80832F5F3F4FDB0151
:10095000CA0180709070AF70B070CD01AA27BB271C
:100960008A30910514F0895C01C0805DF901E2587C
:10097000FB4F80832F5F3F4FDB01CA018070907F68
:10098000A070B070FCE0B695A79597958795FA95FD
:10099000D1F78A30910514F0895C01C0805DF901BE
:1009A000E258FB4F80832F5F3F4FDB01CA0180700D
:1009B0009F70A070B070892F9A2FAB2FBB278A3001
:1009C000910514F0895C01C0805DF901E258FB4F8C
:1009D00080832F5F3F4FDB01CA01807F9070A07042
:1009E000B07074E0B695A795979587957A95D1F7ED
:1009F0008A30910514F0895C01C0805DF901E258EC
:100A0000FB4F80832F5F3F4F4F7050704A3051052E
:100A100014F0495C01C0405DF901E258FB4F40838E
:100A20002F5F3F4FF901E258FB4F80E280832F5F39
:100A30003F4FC9010895DC01FC01E25AFE4FE081FD
:100A40008E2F80538A3038F08151863010F080E04C
:100A500002C08E2F8753982F9295907FA25ABE4F37
:100A60001196EC918E2F80538A3010F4892B0895C3
:100A70008E2F8154863010F080E008958E2F87539A
:100A8000892B0895FC0150814181A82FFC0170E061
:100A900062507040B0E131E416C0228190E0852FB1
:100AA000880F47FD8F5F440F27FD4F5F57FD02C042
:100AB000582F03C0582F5B2743279F5F983011F0B2
:100AC000220FEDCF31968E2F8A1B90E08617970765
:100AD00024F3952F80E0242F30E0282B392BC901F7
:100AE00008952F923F924F925F926F927F928F92D2
:100AF0009F92AF92BF92CF92DF92EF92FF920F93AD
:100B00001F93DF93CF93CDB7DEB728970FB6F89436
:100B1000DEBF0FBECDBF80911E048B3E09F055C1D4
:100B200080911F04803909F050C1809120048B3ED0
:100B300009F04BC180912104803909F046C18091B0
:100B400022048B3E09F041C180912304803909F0D1
:100B50003CC183E096E09C838B83EBE2F6E0FA8372
:100B6000E9836FE3262E66E0362E53E5652E56E0C8
:100B7000752E47E6842E46E0942E3BE7A32E36E002
:100B8000B32E25E8C22E26E0D22E9FE8E92E96E06D
:100B9000F92E01E216E069E976E043EA56E02DEA33
:100BA00036E087E196E098878F83A7EBB6E0E1EC2B
:100BB000F6E0FE83ED8388E0482E512CEB81FC812A
:100BC00080899189938B828BE981FA8180899189CF
:100BD000938B828BF10180899189938B828BF301B6
:100BE00080899189938B828BF40180899189938B81
:100BF000828BF50180858187F60180858187F701E9
:100C000080858187F80180858187FB0180858187C8
:100C1000FA0180858187F90180858187EF81F885D8
:100C20008085818718968C91189719968C931997BF
:100C3000ED81FE8180899189938B828B0894410894
:100C400051088B819C8102979C838B83E981FA8177
:100C50003297FA83E9838EEF9FEF280E391E680ED4
:100C6000791E880E991E0894A108B1080894C1083D
:100C7000D1080894E108F10801501040615070401B
:100C80004150504021503040EF81F8853197F8872E
:100C9000EF8311978D819E8102979E838D839FEFB5
:100CA00049169FEF590609F089CF9091280480E0FA
:100CB0002091270430E0822B932B9093040680939D
:100CC000030690912A0480E02091290430E0822BD1
:100CD000932B90932C0680932B0690912E0480E00A
:100CE00020912D0430E0822B932B9093400680932B
:100CF0003F069091300480E020912F0430E0822B59
:100D0000932B90935406809353069091320480E085
:100D10002091310430E0822B932B909368068093CE
:100D200067068091330480937B068091340480931E
:100D300085068091350480938F06809136048093D8
:100D4000210680913704809399068091380480931E
:100D5000A306809139048093AD0680913A04809374
:100D6000170680913B048093B70690913D0480E084
:100D700020913C0430E0822B932B9093C206809309
:100D8000C10610913F04009140041092400410925B
:100D90003F0484E294E06DE10E94420510933F0419
:100DA0000093400490934204809343048091EC05A7
:100DB0009091ED0501969093ED058093EC051092CE
:100DC000B1051092B00510927E0428960FB6F894E3
:100DD000DEBF0FBECDBFCF91DF911F910F91FF906E
:100DE000EF90DF90CF90BF90AF909F908F907F90CB
:100DF0006F905F904F903F902F90089580EF95E017
:100E00000E948D2C08950F931F93CF93DF938C0135
:100E1000C0E0D0E0F801EC0FFD1F8AEB97E06081A5
:100E20004AE050E00E944C33C330D10531F08AEBE8
:100E300097E060E071E00E94EE332196C430D10566
:100E400049F7DF91CF911F910F910895AC0180EF89
:100E500095E06EE571E022EE32E00E943D2D0895AE
:100E6000EF92FF920F931F93AC0100EF15E07EE528
:100E7000E72E71E0F72EC801B70124EF32E00E949F
:100E80003D2DAC01C801B70123E233E00E943D2DA6
:100E90001F910F91FF90EF90089580EF95E06EE520
:100EA00071E040E050E02DE433E00E943D2D0895D4
:100EB0008EE480937C0062E070E080E090E00E942D
:100EC000A32E80917A00806480937A0080917A00CA
:100ED00086FDFCCF8091780090E0A0E0B0E06091CA
:100EE0007900362F20E0442737FD4095542F282BDA
:100EF000392B4A2B5B2B60E070E381E190E00E948C
:100F0000BC34CA01B9010895CF93DF93EC010CC042
:100F10006A3029F48AEB97E00E949D3204C08AEB84
:100F200097E00E94C4312196FE016491662381F707
:100F3000DF91CF9108950F931F93CF93DF938C018F
:100F4000E091AA05EE2309F400C12091A605222311
:100F500069F48091A705882349F48091A805882326
:100F600029F48091A905882309F4EFC040E0A0E0AE
:100F70008A2F90E0880F991F50E04E1708F451E037
:100F8000A52FA82B4F5F483099F760E0862F90E09F
:100F9000880F991F50E04E1708F451E0652F682B19
:100FA0004F5F403199F770E0872F90E0880F991FCD
:100FB00050E04E1708F451E0752F782B4F5F483101
:100FC00099F780E090E0880F991F50E04E1708F4E1
:100FD00051E0582B852F4F5F4032A1F7F801E25ABC
:100FE000FE4F8081C82FD0E08A2F90E08C239D2374
:100FF00030E08217930729F5862F90E0218130E0B9
:10100000822393232091A70530E082179307C9F428
:10101000872F90E0228130E0822393232091A8053E
:1010200030E08217930769F4852F90E0238130E048
:10103000822393232091A90530E08217930709F4B6
:1010400084C0E091AF05EE2309F47CC02091AB058C
:10105000222369F48091AC05882349F48091AD0581
:10106000882329F48091AE05882309F46BC0F72FFB
:1010700040E08F2F90E0880F991F50E04E1708F442
:1010800051E0F52FF82B4F5F483099F7672F862FE7
:1010900090E0880F991F50E04E1708F451E0652F3B
:1010A000682B4F5F403199F7872F90E0880F991F89
:1010B00050E04E1708F451E0752F782B4F5F483100
:1010C00099F750E0852F90E0880F991F50E04E1758
:1010D00008F451E0A52FA82B5A2F4F5F403291F70B
:1010E0008F2F90E08C239D2330E08217930751F5DA
:1010F000862F90E0F801E25AFE4F218130E08223F2
:1011000093232091AC0530E082179307D9F4872F01
:1011100090E0228130E0822393232091AD0530E0DE
:101120008217930779F4C0E0D0E08A2F90E0238102
:1011300030E0822393232091AE0530E0821793079D
:1011400031F403C0C0E0D0E002C0C1E0D0E0809143
:10115000B4059091B505892B31F0209721F489E8E9
:1011600092E00E948407CE01DF91CF911F910F91F1
:10117000089580915C0190915D01039781F482E074
:1011800090E090935D0180935C018091B405909113
:10119000B505892B21F088EA92E00E948407089522
:1011A000AF92BF92CF92DF92EF92FF920F931F9375
:1011B000CF93DF935C014091FF05509100064115EC
:1011C000510579F0C0910106D0910206FE01EE0FA3
:1011D000FF1FE856FF4F659174910E946203892BAF
:1011E00019F1CC24DD24E7E1EE2EF12CE601CE0D41
:1011F000DF1DD595C795D0930206C0930106FE0169
:10120000EE0FFF1FE856FF4F05911491C8010E9491
:101210005903AC01909300068093FF05C501B80106
:101220000E946203009719F4FE01B09611C01816CF
:1012300019062CF46E010894C11CD11C04C07E0157
:101240000894E108F108EC14FD0484F6E0E0F0E015
:10125000CF01DF91CF911F910F91FF90EF90DF9021
:10126000CF90BF90AF900895CF92DF92EF92FF9210
:101270000F931F93CF93DF93C0905C01D0905D01DB
:101280000E949F2D029709F0E2C00E94952E2091A6
:10129000C8053091C9054091CA055091CB05621B24
:1012A000730B840B950B615A7B4B8D40904008F477
:1012B000CEC080915C0190915D01181619060CF06A
:1012C000C6C08091EC059091ED0509970CF4BFC064
:1012D0000E94952E6093C8057093C9058093CA0536
:1012E0009093CB05C091EC05D091ED05CB30D105A5
:1012F00014F0CAE0D0E0E3E0F6E060E070E020E067
:1013000030E040E050E00AC081919191A0E0B0E06F
:10131000280F391F4A1F5B1F6F5F7F4F6C177D07B8
:101320009CF3CA01B9012AE030E040E050E00E949D
:1013300054349E01442737FD4095542F0E949A341F
:1013400079018A0120E030E040E050E008C0F90176
:10135000E95EF94F8081480F511D2F5F3F4F2C17D9
:101360003D07ACF320E030E060E070E008C0F90138
:10137000EF5DF94F8081680F711D2F5F3F4F2C1774
:101380003D07ACF380914C0190914D01A0E0B0E09D
:10139000E816F9060A071B07A8F04C175D0791F439
:1013A00080915001909151019C01429FC001439F47
:1013B000900D529F900D11246817790718F081E065
:1013C000C82ED12C80914E0190914F01A0E0B0E049
:1013D000E816F9060A071B0788F0452B79F080917B
:1013E0005201909153019C01C29FC001C39F900D77
:1013F000D29F900D11246817790748F580915C0100
:1014000090915D01019719F51092E4051092E505A0
:101410001092E6051092E7051092E0051092E105A2
:101420001092E2051092E3051092DC051092DD05A2
:101430001092DE051092DF051092D8051092D905A2
:101440001092DA051092DB0502E0C02ED12C8091BB
:101450005C0190915D01039709F062C08091D40511
:101460009091D505A091D605B091D705805C944D9B
:10147000A140B04008F454C00E94952E2091CC05A4
:101480003091CD054091CE055091CF05621B730B75
:10149000840B950B2091D4053091D5054091D6054C
:1014A0005091D705220F331F441F551F26173707AA
:1014B00048075907A8F51092E4051092E505109227
:1014C000E6051092E7051092E0051092E1051092F2
:1014D000E2051092E3051092DC051092DD051092F2
:1014E000DE051092DF051092D8051092D9051092F2
:1014F000DA051092DB0580EF95E00E94912C0E94A6
:10150000952E6093D0057093D1058093D20590936A
:10151000D3051092E9051092E805B2E0CB2ED12C4C
:10152000C601DF91CF911F910F91FF90EF90DF9057
:10153000CF9008950E949F2D805D80937E048091BE
:10154000EC059091ED05409734F08FE090E090939A
:10155000ED058093EC058091EC059091ED058A30C6
:10156000910514F0895C01C0805D80937F048091B7
:101570005C01805D809380048091E805805D8093AC
:10158000810480E2809382040E94DA2DAB01BC01C9
:1015900085E090E00E94620408950E944D070E9439
:1015A0003007AC0180EF95E06EE571E02EE734E0A6
:1015B0000E94372D0E9426070895EF92FF920F9305
:1015C0001F93CF93DF937C010E94DA2D0E949F2D01
:1015D000805D80937E048091EC059091ED054097AD
:1015E00034F08FE090E09093ED058093EC058091CE
:1015F000EC059091ED058A30910514F0895C01C0ED
:10160000805D80937F0480915C01805D8093800485
:101610008091E805805D8093810480E2809382045C
:101620000E94DA2DAB01BC0185E090E00E946204CB
:10163000FC011E141F0434F5CEE1D4E0DC01A258F5
:10164000BB4F20E29881892F82958F708A3010F0ED
:10165000895C01C0805D8C93892F8F708A3010F077
:10166000895C01C0805D11968C93119712962C9322
:1016700012972196139684E0C634D80719F7E858D4
:10168000FF4F6DC06091EC057091ED0516161706C1
:101690000CF065C0EB016B30710514F0CAE0D0E0CE
:1016A000CF01BE0143E056E00E94E203BE014BE2DF
:1016B00056E00E94E203BE014FE356E00E94E203BF
:1016C000BE0143E556E00E94E203BE0147E656E054
:1016D0000E94E203BE0141EC56E00E94E203BE011B
:1016E00040E050E02BE736E00E948503BE0140E079
:1016F00050E025E836E00E948503BE0140E050E05E
:101700002FE836E00E948503BE0141E050E021E26F
:1017100036E00E948503BE0140E050E029E936E052
:101720000E948503BE0140E050E023EA36E00E94BB
:101730008503BE0140E050E02DEA36E00E948503BB
:10174000BE0140E050E027E136E00E948503BE0183
:1017500041E050E027EB36E00E948503FC01F09366
:10176000B305E093B205E258FB4F10828EE591E09D
:101770000E94CD0A182F092F8091B4059091B505CC
:101780001816190694F48CED92E00E94840760917B
:10179000B0057091B1058AEB97E04AE050E00E94F5
:1017A000BC338FEC92E00E948407EF2821F4109262
:1017B000ED051092EC05812F902FDF91CF911F91B5
:1017C0000F91FF90EF9008955F926F927F928F92AA
:1017D0009F92AF92BF92CF92DF92EF92FF920F93C0
:1017E0001F93CF93DF933C010E949A0AEC0185E19D
:1017F0000E94412FAA24BB24812C24E0922E00E0D9
:1018000010E0CC24DD24760190E2592E64E170E0F2
:1018100080E090E00E94A32E85E10E94412F9C0170
:10182000881599050CF44C01021713070CF4890173
:101830006114710429F084E0A816B10409F047C0CE
:10184000E3E0293E3E0764F0FE01E258FB4FC90188
:1018500068EE73E00E948734605D6083219603C068
:101860002536310584F0FE01E258FB4FC90168EED0
:1018700073E00E94873464E670E00E948734605D04
:101880006083219603C02B3031057CF0FE01E258C5
:10189000FB4FC90164E670E00E9487346AE070E0A3
:1018A0000E948734605D60832196FE01E258FB4F01
:1018B000C9016AE070E00E948734805D8083CE01B8
:1018C0000196FC01E258FB4F5082EC012196C901C0
:1018D000AA2797FDA095BA2FC80ED91EEA1EFB1E97
:1018E0000894A11CB11CF7E0AF16B10409F08ECF2B
:1018F000080D191DC801AA2797FDA095BA2FC81A6F
:10190000D90AEA0AFB0AA0904A01B0904B0195015E
:1019100040E050E0C701B6010E94543420E034E1B9
:1019200040E050E00E949A3469017A01FE01E258D9
:10193000FB4F88E28083219681E1C81687E2D806B2
:1019400080E0E80680E0F80680F08E0102581B4F28
:10195000C701B60120E137E240E050E00E949A342E
:10196000205DF8012083219609C0F9EECF16F3E03F
:10197000DF06F0E0EF06F0E0FF06B0F08E0102585F
:101980001B4FC701B60120E137E240E050E00E9462
:101990009A3428EE33E040E050E00E949A34205D13
:1019A000F8012083219606C0F5E6CF16D104E104A4
:1019B000F104B0F08E0102581B4FC701B60128EEAA
:1019C00033E040E050E00E949A3424E630E040E00A
:1019D00050E00E949A34205DF8012083219606C0D1
:1019E000FBE0CF16D104E104F104A8F08E01025807
:1019F0001B4FC701B60124E630E040E050E00E94F2
:101A00009A342AE030E040E050E00E949A34205DB1
:101A1000F801208321968E0102581B4FC701B601A1
:101A20002AE030E040E050E00E949A34605DF80126
:101A30006083CE010196FC01E258FB4F30E2308317
:101A40000196FC01E258FB4F2DE620830196FC0134
:101A5000E258FB4F26E520830196FC01E258FB4F3C
:101A600029E22083DC011196672809F47DC0FD017D
:101A7000E258FB4F3083CD010196FC01E258FB4F49
:101A80002DE420830196FC01E258FB4F21E62083E0
:101A90000196FC01E258FB4F28E720830196FC01E8
:101AA000E258FB4F2AE320839C012F5F3F4FF1E177
:101AB000AF16F7E2BF0668F0F901E258FB4FC50127
:101AC00060E177E20E947334605D60832F5F3F4F77
:101AD00005C089EEA81683E0B80688F0F901E2583F
:101AE000FB4FC50160E177E20E94733468EE73E05A
:101AF0000E947334605D60832F5F3F4F04C0E5E652
:101B0000AE16B10488F0F901E258FB4FC50168EE4A
:101B100073E00E94733464E670E00E947334605D89
:101B200060832F5F3F4F04C0FBE0AF16B10480F02D
:101B3000F901E258FB4FC50164E670E00E9473347E
:101B40006AE070E00E947334605D60832F5F3F4FF6
:101B5000F901E258FB4FC5016AE070E00E9473345E
:101B6000805D8083D9011196A258BB4F1C928EE5EF
:101B700091E00E94CD0ADF91CF911F910F91FF90CC
:101B8000EF90DF90CF90BF90AF909F908F907F901D
:101B90006F905F9008950F931F93DF93CF9300D0C2
:101BA000CDB7DEB70E949A0AFC01E258FB4F26E44B
:101BB00020830196FC01E258FB4F22E72083019627
:101BC000FC01E258FB4F25E620830196FC01E25818
:101BD000FB4F20830196FC01E258FB4F2AE3208350
:101BE0000196FC01E258FB4F20E220838C010F5F3D
:101BF0001F4F8091EC079091ED07009711F480EF53
:101C000097E09E012F5F3F4F281B390B87E2203161
:101C1000380718F020E030E038C083E0293E38076C
:101C20006CF0F801E258FB4FC90168EE73E00E94C6
:101C30008734605D60830F5F1F4F03C02536310519
:101C40008CF0F801E258FB4FC90168EE73E00E9486
:101C5000873464E670E00E948734605D60830F5FC4
:101C60001F4F03C02B30310584F0F801E258FB4FC1
:101C7000C90164E670E00E9487346AE070E00E9467
:101C80008734605D60830F5F1F4FF801E258FB4FA0
:101C9000C9016AE070E00E948734805D8083F801AA
:101CA0003196DF01A258BB4F80E28C933196DF0161
:101CB000A258BB4F82E68C933196DF01A258BB4FEE
:101CC00089E78C933196DF01A258BB4F84E78C9350
:101CD0003196DF01A258BB4F85E68C93E158FB4F4C
:101CE00083E7808311828EE591E00E94CD0A0F90F8
:101CF0000F90CF91DF911F910F9108950F931F9334
:101D00008C010E949A0AA80160E070E00E946204BF
:101D1000FC01E258FB4FAC014F5F5F4F04311105EE
:101D200048F08FE48083FA01E258FB4F8BE4808314
:101D3000FA010EC085E48083FA01E258FB4F22E5E8
:101D40002083CA010196FC01E258FB4F2083FC016D
:101D50003196E258FB4F10828EE591E00E94CD0A49
:101D60001F910F9108950F931F930E949A0A8C015F
:101D70000E94DA2DAB01BC018091B8059091B905A4
:101D8000A091BA05B091BB05481B590B6A0B7B0BA0
:101D9000C8010E946204FC019093B3058093B205D0
:101DA000E258FB4F10828EE591E00E94CD0A1F9110
:101DB0000F9108957F928F929F92AF92BF92CF9290
:101DC000DF92EF92FF920F931F93CF93DF93EC017B
:101DD000672B09F4D1C082E091E0BE0144E050E0FD
:101DE0000E947703009709F0C7C0FC8005E010E06F
:101DF000AA24BB2465011DC0C601B5012AE030E05C
:101E000040E050E00E9454342F2D332727FD3095B9
:101E1000205330405901CC24B7FCC094DC2CA60ED2
:101E2000B71EC81ED91EFE01E00FF11FF0800F5F24
:101E30001F4F8F2D80538A3018F40F301105E1F6B3
:101E4000B801615070406C0F7D1F87E091E044E065
:101E500050E00E947703009721F0EE24FF248701D1
:101E600047C0FE01E00FF11F738044E0842E912CE7
:101E7000800E911EEF01EE24FF2487011BC0C801D4
:101E8000B7012AE030E040E050E00E945434272DB2
:101E9000332727FD30952053304079010027F7FC88
:101EA0000095102FE60EF71E081F191F7B8008945F
:101EB000811C911C872D80538A3028F4219629E1BA
:101EC00082169104E4F2D801C70188579040A040DF
:101ED000B040895A9B41A040B04030F030EBE32E37
:101EE00034E0F32E012D112DC801B7010E94A42D5D
:101EF0000E949F2D892BB1F40E94952E28EE33E08D
:101F000040E050E00E949A34D601C501821B930B39
:101F1000A40BB50B8093B8059093B905A093BA05AF
:101F2000B093BB05C601B5010E94AD2D8091B405EB
:101F30009091B505892B01F18EE992E00E9484070A
:101F40008AEB97E0B601A5012AE030E00E943D331C
:101F50008AEB97E06CE071E00E94EE338AEB97E049
:101F6000B801A7012AE030E00E943D338AEB97E0F8
:101F70006EE071E00E94F1330E94B30EDF91CF91C9
:101F80001F910F91FF90EF90DF90CF90BF90AF9097
:101F90009F908F907F900895CF92DF92EF92FF9263
:101FA0000F931F93CF93DF9391E090937E048093E0
:101FB0007F0460938004A5EDB6E0C1E8D4E0E62F8D
:101FC000F0E09F012A0F3B1F02C08D918993A21759
:101FD000B307D9F771E8E72E74E0F72EEE0EFF1E77
:101FE000D7011C928F010E571B4FD8011C9255E050
:101FF000C52ED12CCE0EDF1EF601E258FB4F8FE727
:1020000080836B5F8EE794E00E944205F701908326
:10201000D8018C93C0E0D0E08091EE059091EF055F
:10202000892B89F08091B4059091B505892B59F4DD
:102030008AEB97E06BEE0E94C4318AEB97E060E98F
:102040000E94C4311AC08AEB97E06BEE70E040E169
:1020500050E00E94BC338AEB97E060E20E94953228
:102060008AEB97E060E970E040E150E00E94BC3309
:102070008AEB97E060E20E9495322196C330D10549
:1020800059F6CEE7D4E000E010E08091EE059091A3
:10209000EF05892B51F08091B4059091B505892BFE
:1020A00021F48AEB97E0688112C08881803128F49E
:1020B0008AEB97E060E30E9495328AEB97E06881B3
:1020C00040E150E00E944C338AEB97E060E20E94CE
:1020D000C4310F5F1F4F2196C016D106B4F6809110
:1020E000EE059091EF05892B39F08091B405909120
:1020F000B5051816190624F48AEB97E00E949D3264
:10210000DF91CF911F910F91FF90EF90DF90CF90D3
:1021100008951092D506892B19F081E08093D50699
:102120001092D6068AEA61E00E94CC0F0895CF9300
:10213000DF93C0E0D0E088E197E0BE010E948C2DE3
:10214000FE01E25EFB4F80832196C034D10599F7F2
:1021500010925E0480911E048D34A9F580911F04B5
:10216000813489F55091200440912104309122045A
:10217000209123049091240480912504552359F43F
:102180004423A9F4332399F4222389F4992379F47D
:10219000882369F418C05F3F51F44F3F41F43F3F3B
:1021A00031F42F3F21F49F3F11F48F3F61F05093A2
:1021B0002F014093300130933101209332019093ED
:1021C00033018093340180912604813421F580917C
:1021D0002704843401F5809128048434E1F480914B
:1021E00029048235C1F430912A0420912B04909166
:1021F0002C0480912D043F3F31F42F3F21F49F3F69
:1022000011F48F3F41F030933501209336019093C4
:1022100037018093380180913604873469F58091C5
:102220003704813449F580913804843529F580914B
:102230003904853409F530913A0420913B0490919A
:102240003C0480913D04332339F4222369F499231B
:1022500059F4882349F410C03F3F31F42F3F21F453
:102260009F3F11F48F3F41F03093390120933A01A1
:1022700090933B0180933C0180913E048035B1F402
:1022800080913F048F3491F480914004823571F441
:1022900080914104843551F480914204909143042B
:1022A000882311F4992311F09093490180914404FB
:1022B000813409F073C080914504833409F06EC005
:1022C00080914604833409F069C0809147048133CA
:1022D00009F064C0409148043091490420914A04B7
:1022E00090914B0450914C04852F8150803208F01E
:1022F00055C0442339F4332371F4222361F4992324
:1023000051F44CC04F3F39F43F3F29F42F3F19F4AB
:102310009F3F09F443C04093A6053093A70520933F
:10232000A8059093A9055093AA0580914D04813486
:10233000A9F580914E04833489F580914F0483344C
:1023400069F580915004823349F5409151043091F0
:102350005204209153049091540450915504852FB8
:1023600081508032D8F4442339F4332369F4222392
:1023700059F4992349F412C04F3F31F43F3F21F4FF
:102380002F3F11F49F3F51F04093AB053093AC05C4
:102390002093AD059093AE055093AF058091560400
:1023A0008234E1F4809157048635C1F48091580459
:1023B0008934A1F4809159048E3481F420915A0417
:1023C00030915B04222311F4332341F0922F80E0FB
:1023D000830F911D90934B0180934A018091620479
:1023E0008335E1F4809163048435C1F48091640401
:1023F0008234A1F4809165048C3481F420916604C8
:1024000030916704222311F4332341F0922F80E0AE
:10241000830F911D90934F0180934E01809168042A
:102420008335E1F4809169048F34C1F480916A04AA
:102430008334A1F480916B04883481F420916C047E
:1024400030916D04222311F4332341F0922F80E068
:10245000830F911D909351018093500180916E04E0
:102460008335E1F480916F048F34C1F4809170045E
:102470008334A1F4809171048C3481F4209172042E
:1024800030917304222311F4332341F0922F80E022
:10249000830F911D9093530180935201DF91CF914F
:1024A00008954F925F926F927F928F929F92AF9218
:1024B000BF92CF92DF92EF92FF920F931F93DF9321
:1024C000CF9300D0CDB7DEB782E060E00E94632FEB
:1024D00089E061E00E94632F82E00E94F62F01975D
:1024E00011F40E94971085E10E94412F10E06624AC
:1024F00077246AE070E080E090E00E94A32E85E1FE
:102500000E94412F680E791E1F5F153091F7409091
:102510004A0150904B0189EF681681E0780634F04B
:1025200081E090E09093EF058093EE058AEB97E0D1
:1025300040E855E260E070E00E94D3308AEB97E01B
:102540000E9404328823D1F387E691E00E94840739
:1025500080EF95E00E94892D80EF95E00E94912CFC
:1025600080E592E00E94840780EF95E06FE271E0E1
:102570000E94852D8AE492E00E94840788E392E01D
:102580000E94840780EF95E00E94492D682F8AEB16
:1025900097E040E150E00E945E3380EF95E00E94BA
:1025A000492D882321F48DE192E00E9484078091D7
:1025B0003501882309F065C080913601882309F030
:1025C00060C080913701882309F05BC08091380199
:1025D000882309F056C08091EE059091EF05892B74
:1025E00021F482E092E00E94840700D08DE391E024
:1025F000EDB7FEB79283818380EF95E06EE571E0E1
:1026000040EC52E02FE231E000E510E0B5E3EB2EC4
:10261000B1E0FB2EA5E4CA2EA1E0DA2EF9E3AF2E3D
:10262000F1E0BF2EE1E48E2EE1E09E2E0E949E2C72
:102630000F900F902091EE053091EF05882339F02F
:10264000232BF9F48CEF91E00E9484071AC0232B0E
:1026500021F486EE91E00E94840730EC309335013E
:1026600028EA2093360191E09093370189E1809325
:1026700038013093390120933A0190933B019093B4
:102680003C012091490180EF95E06FE271E045E364
:1026900051E030E00E94432D80EF95E069E371E066
:1026A0000E942E2D88ED91E00E9484078091EC0716
:1026B0009091ED07009711F480EF97E0BE016F5FF6
:1026C0007F4F681B790B8AEB97E04AE050E00E944D
:1026D000BC338AEC91E00E9484070E945807AB014A
:1026E000BC018AEB97E02AE030E00E947C338FEB5C
:1026F00091E00E948407B301882777FD8095982F89
:10270000920140E050E00E94543420E034E140E087
:1027100050E00E949A348AEB97E0BA01A9012AE0BE
:1027200030E00E943D338AEB91E00E948407809163
:10273000EE059091EF05892BE1F48DEA91E00E947E
:10274000840785E391E00E94030781EA91E00E94FB
:10275000840785E491E00E94030785E991E00E94E7
:10276000840789E391E00E9403078AEB97E00E94C7
:102770009D321092B3051092B2051092B1051092DD
:10278000B0051092E4051092E5051092E60510924E
:10279000E7051092E0051092E1051092E205109213
:1027A000E3051092DC051092DD051092DE05109213
:1027B000DF051092D8051092D9051092DA05109213
:1027C000DB050E94952E6093D0057093D105809310
:1027D000D2059093D3056093CC057093CD0580937B
:1027E000CE059093CF0581E090E00E948910109271
:1027F000E9051092E80581E090E09093EB05809365
:10280000EA050F900F90CF91DF911F910F91FF90EC
:10281000EF90DF90CF90BF90AF909F908F907F9080
:102820006F905F904F9008955F926F927F928F921A
:102830009F92AF92BF92CF92DF92EF92FF920F934F
:102840001F93CF93DF937C010E944D070E943007B6
:102850006C01F694FE2CEE24F794E7948F2D8F7084
:102860008A3010F0895C01C0805D80937E04C701CE
:10287000B4E096958795BA95E1F78870805D80936E
:102880007F0480E3809380048AE38093810480E264
:10289000809382048701C5E0D0E0A0E8AA2EB12C85
:1028A000AE0CBF1CFDE05F2EEAE06E2E70E3772ECB
:1028B0006AE3862E50E2952E84C0E016F1060CF0F5
:1028C00057C0C8018F709070892B09F051C0FE016C
:1028D000E258FB4F5082CE010196FC01E258FB4FBB
:1028E00060829C012F5F3F4F812F8F708A3010F0E4
:1028F000895C01C0805DF901E258FB4F80832F5F46
:102900003F4FC801807F907044E0959587954A9528
:10291000E1F78A3010F0895C01C0805DF901E2586E
:10292000FB4F8083C9010196FC01E258FB4F708286
:102930000196FC01E258FB4F80820196FC01E258AF
:10294000FB4F9082EC012196C8018F739070892B08
:1029500079F4C258DB4F188280EF95E06EE571E0A4
:10296000A6012EE734E00E94372D6C01C0E0D0E0D4
:1029700088E197E0B8010E948C2D982F92959F7066
:10298000282F2F709A3018F0892F895C02C0892F68
:10299000805DFE01E258FB4F8083CE0101962A3014
:1029A00010F0295C01C0205DFC01E258FB4F208340
:1029B0000196FC01E258FB4F9082EC0121960F5FDB
:1029C0001F4F0A151B0509F078CFC258DB4F18823C
:1029D00080EF95E06EE571E0A6012EE734E00E94FD
:1029E000372D0E942607DF91CF911F910F91FF9005
:1029F000EF90DF90CF90BF90AF909F908F907F909F
:102A00006F905F900895CF92DF92EF92FF920F93B5
:102A10001F93CF93DF938C017B01EA01690188E169
:102A200097E06EE370E043E50E94932D88E197E024
:102A30006FE370E044E50E94932D88E197E060E445
:102A400070E042E40E94932D88E197E061E470E039
:102A500048E40E94932D88E197E062E470E0412F02
:102A60000E94932D88E197E063E470E0402F0E947C
:102A7000932D88E197E064E470E043E50E94932D94
:102A800088E197E065E470E044E50E94932D88E1D9
:102A900097E066E470E042E40E94932D88E197E0BD
:102AA00067E470E04CE40E94932D88E197E068E4CD
:102AB00070E04F2D0E94932D88E197E069E470E06B
:102AC0004E2D0E94932D209709F45FC01C141D0405
:102AD0000CF05BC0CC16DD0608F057C088E197E02B
:102AE0006AE470E043E50E94932D88E197E06BE48F
:102AF00070E04FE40E94932D88E197E06CE470E071
:102B000043E40E94932D88E197E06DE470E048E48F
:102B10000E94932D88E197E06EE470E04D2F0E94B3
:102B2000932D88E197E06FE470E04C2F0E94932D85
:102B300088E197E060E570E043E50E94932D88E12D
:102B400097E061E570E04FE40E94932D88E197E003
:102B500062E570E043E40E94932D88E197E063E52D
:102B600070E04CE40E94932D4D2D552747FD5A955A
:102B700088E197E064E570E00E94932D88E197E09A
:102B800065E570E04C2D0E94932DDF91CF911F9150
:102B90000F91FF90EF90DF90CF9008954F925F924A
:102BA0006F927F928F929F92AF92BF92CF92DF925D
:102BB000EF92FF920F931F93CF93DF933C0182E03C
:102BC00091E0B30144E050E00E947703009709F0E0
:102BD0002FC1F3011481C5E0D0E088249924540169
:102BE0001CC0C501B4012AE030E040E050E00E9482
:102BF0005434212F332727FD30952053304049018D
:102C0000AA2497FCA094BA2C860E971EA81EB91E63
:102C1000F301EC0FFD1F10812196812F80538A3024
:102C200018F4CA30D105E9F6BE0161507040660D56
:102C3000771D87E091E044E050E00E947703009721
:102C400009F0F6C0F301EC0FFD1F53808E010C5FFD
:102C50001F4FEF01CC24DD2476011AC0C701B60155
:102C60002AE030E040E050E00E945434252D332724
:102C700027FD3095205330406901EE24D7FCE094C5
:102C8000FE2CC60ED71EE81EF91E5B800F5F1F4F7D
:102C9000852D80538A3020F4219605311105F4F2F8
:102CA000B80161507040660D771D80E191E044E00D
:102CB00050E00E947703009709F07DC0A8014A5FA9
:102CC0005F4FF301E00FF11F2381E8012496F30128
:102CD000E00FF11F00E010E014C0C801B3E0880F5E
:102CE000991FBA95E1F7000F111F080F191F822FC6
:102CF000992787FD9095080F191F005310402381D5
:102D00002196822F80538A3020F431964C175D072C
:102D100024F72801BE0161507040660D771D85E1E2
:102D200091E044E050E00E947703009719F020E022
:102D300030E02CC0DE011696F301EC0FFD1F63811D
:102D4000AE014C5F5F4FF301EC0FFD1F20E030E060
:102D500015C0C90173E0880F991F7A95E1F7220F1A
:102D6000331F280F391F862F992787FD9095280F2D
:102D7000391F2053304063814F5F5F4F862F805350
:102D80008A3020F43196A417B5071CF704361105D4
:102D900094F4201731077CF40333110564F02932D1
:102DA00031054CF0109351010093500130935301C1
:102DB0002093520104C04424552420E030E0C8147C
:102DC000D904EA04FB04A0F5F8E38F16F1E39F06AB
:102DD000F0E0AF06F0E0BF0658F181E488168AE61D
:102DE000980680E0A80680E0B80610F5E0E7CE1669
:102DF000E0E3DE06E0E0EE06E0E0FE06C8F0F1E922
:102E0000CF16F5E6DF06F0E0EF06F0E0FF0680F40F
:102E100090924D0180924C01D0924F01C0924E0190
:102E2000C401B601A2010E940315C1E0D0E002C0B6
:102E3000C0E0D0E00E944D070E943007AC01CD2BCE
:102E400049F08FE480937E048BE680937F04E2E078
:102E5000F0E00AC085E480937E0482E780937F04DB
:102E600080938004E3E0F0E0E258FB4F8AE0808347
:102E7000118280EF95E06EE571E02EE734E00E946C
:102E8000372D0E942607DF91CF911F910F91FF9060
:102E9000EF90DF90CF90BF90AF909F908F907F90FA
:102EA0006F905F904F900895EF92FF920F931F9352
:102EB0007C0108E117E0C80168E370E042E40E9489
:102EC000932DC80169E370E046E50E94932DC80187
:102ED0006AE370E049E40E94932DC8016BE370E05F
:102EE0004EE40E94932D4F2D552747FD5A95C8015A
:102EF0006CE370E00E94932DC8016DE370E04E2DED
:102F00000E94932D1F910F91FF90EF900895BF9213
:102F1000CF92DF92EF92FF920F931F93CF93DF93A5
:102F20006C0182E091E0B60144E050E00E9477033A
:102F3000009709F049C0F601B480C5E0D0E0EE2466
:102F4000FF2487011CC0C801B7012AE030E040E03F
:102F500050E00E9454342B2D332727FD3095205309
:102F6000304079010027F7FC0095102FE60EF71E80
:102F7000081F191FF601EC0FFD1FB08021968B2D45
:102F800080538A3018F4CA30D105E9F6D801C70158
:102F9000815A9F40A040B04080569D46A040B0401E
:102FA00098F4F0924B01E0924A012197CC0DDD1D7F
:102FB0008AE191E0BE0145E050E00E94770300976E
:102FC00019F4C7010E94541781E090E00E94E40BBD
:102FD000DF91CF911F910F91FF90EF90DF90CF90F5
:102FE000BF9008956F927F928F929F92AF92BF92FF
:102FF000CF92DF92EF92FF920F931F93CF93DF93C5
:103000006C01EB01625A7E4F82E091E044E050E0B7
:103010000E947703009709F0D2C1CE0104960E9466
:103020001B05782E26E0E22EF12CEC0EFD1EC701CA
:103030000E941B05682E80E2C816D10419F488246A
:10304000992419C0CE0108960E941B05882E9AE08B
:10305000E92EF12CEC0EFD1EC7010E941B05982ED7
:10306000C114D10451F096E2C916D10431F08FE2B7
:10307000C816D10411F0AA240BC082E090E0E80E3B
:10308000F91EC7010E941B05A82EC114D10411F01E
:10309000BB2408C082E090E0E80EF91EC7010E9440
:1030A0001B05B82E8091B4059091B505892B09F4C4
:1030B00043C08AEB97E0672D4AE050E00E944C3312
:1030C0008AEB97E06EE20E9495328AEB97E0662DDC
:1030D0004AE050E00E944C338AEB97E06EE20E9497
:1030E00095328AEB97E0682D4AE050E00E944C331D
:1030F0008AEB97E06EE20E9495328AEB97E0692DA9
:103100004AE050E00E944C338AEB97E06EE20E9466
:1031100095328AEB97E06A2D4AE050E00E944C33EA
:103120008AEB97E06EE20E9495328AEB97E06B2D76
:103130004AE050E00E945E3398E0C916D10409F4D9
:1031400045C0772059F4662049F4882039F4992045
:1031500029F4AA2019F4BB2009F43DC188E1C8165E
:10316000D10409F471C099E1C916D1046CF488E066
:10317000C816D10459F190E1C916D10409F445C02B
:10318000C114D10491F00FC086E2C816D10409F42D
:1031900099C09FE2C916D10409F494C080E2C81610
:1031A000D10409F470C0E601BDC088E197E060E099
:1031B00070E04DE40E94932D88E197E061E070E0BB
:1031C00041E40E94932DC2E0D0E0ACC088E197E0DA
:1031D00068E070E041E40E94932D88E197E069E0A7
:1031E00070E044E40E94932D88E197E06AE070E08B
:1031F00044E40E94932D88E197E06BE070E042E5A3
:103200000E94932DCCE0D0E08DC088E197E060E192
:1032100070E04DE40E94932D88E197E061E170E059
:1032200041E40E94932D88E197E062E170E043E57C
:103230000E94932D88E197E063E170E04BE40E94E7
:10324000932DC4E1D0E06EC088E197E068E170E0C2
:1032500047E40E94932D88E197E069E170E041E442
:103260000E94932D88E197E06AE170E044E50E94B6
:10327000932D88E197E06BE170E045E40E94932D87
:10328000CCE1D0E04FC088E197E060E270E040E53B
:103290000E94932D88E197E061E270E04FE40E9484
:1032A000932D88E197E062E270E042E50E94932D61
:1032B00088E197E063E270E044E50E94932DC4E268
:1032C000D0E030C086010F5F1F4F88E197E0B60164
:1032D00041E40E94932D78010894E11CF11C88E1DF
:1032E00097E0B80143E40E94932D87010F5F1F4FC1
:1032F00088E197E0B70143E40E94932DB8016F5F26
:103300007F4F96E2C916D10431F4EB0188E197E0D2
:10331000B80141E305C0EB0188E197E0B80142E361
:103320000E94932D8E010F5F1F4F88E197E0BE0131
:10333000472D0E94932D78010894E11CF11C88E12F
:1033400097E0B801462D0E94932D80E2C816D10463
:1033500009F441C087010F5F1F4F88E197E0B70173
:10336000482D0E94932D78010894E11CF11C88E1FE
:1033700097E0B801492D0E94932DC114D10441F06A
:1033800096E2C916D10421F08FE2C816D10419F5CE
:10339000E701219688E197E0B7014A2D0E94932D1D
:1033A000CD2811F07E0117C07E010894E11CF11CAC
:1033B00088E197E0BE014B2D0E94932D0CC08091B7
:1033C000B4059091B505892B21F08CEB92E00E9419
:1033D0008407EE24FF24C701DF91CF911F910F9145
:1033E000FF90EF90DF90CF90BF90AF909F908F9025
:1033F0007F906F900895AF92BF92DF92EF92FF920D
:103400000F931F93CF93DF93C091F105D091F205F5
:10341000BE01625A7E4FFB019E01AE01405C5F4FD0
:103420000AC09081892F81568A3110F4905290837E
:103430002F5F3F4F31962417350720F482E0213C5F
:10344000380778F380E291E044E050E00E9477038F
:10345000009781F00E944D07AC019093F205809394
:10346000F10580EF95E06EE571E029E732E00E941A
:103470003D2D17C2CE59DE4F85E291E0BE0142E0FC
:1034800050E00E947703009709F442C08091B40590
:103490009091B505892B21F08EE692E00E94840779
:1034A0008091F1059091F2058D599E4F0E94D008B0
:1034B000EC018091B4059091B505892B39F08AEB28
:1034C00097E0BE014AE050E00E94CF33FE01B09782
:1034D000E831F10508F0EAC1EC5CFF4FEE0FFF1F89
:1034E0000590F491E02D099420E030E08091B4053E
:1034F0009091B505892B11F421E030E03093B505AA
:103500002093B405232B21F082E692E00E948407E9
:103510008EE591E00E94CD0AC4C16091F1057091E1
:10352000F205675F7F4F80E090E023C06091F10576
:103530007091F205675F7F4F88E090E01AC060915C
:10354000F1057091F205675F7F4F80E190E011C057
:103550006091F1057091F205675F7F4F88E190E01F
:1035600008C06091F1057091F205675F7F4F80E2BE
:1035700090E00E94F2179DC16091F1057091F205F3
:10358000FB01E25AFE4F8085813329F4675F7F4F4C
:1035900086E290E0EECF823309F08BC1675F7F4F08
:1035A0008FE290E0E6CF1092EB051092EA0581C120
:1035B000C091F105D091F205BE0169597E4F82E0BC
:1035C00091E044E050E00E947703009709F06EC15B
:1035D000C25ADE4F6D85603319F480E090E004C07C
:1035E000613341F581E090E00E94891023C0C091D1
:1035F000F105D091F205BE0166597E4F82E091E05F
:1036000044E050E00E9477030097A1F4C25ADE4FD5
:103610006889603329F410925D0110925C010AC040
:10362000613311F0623331F482E090E090935D01F8
:1036300080935C0181E090E00E94DD0A32C181E06C
:1036400090E002C080E090E00E94DD0A9093F205D5
:103650008093F1050E94952E6093C4057093C50573
:103660008093C6059093C705A3C00091F105109102
:10367000F205E801C459DE4F82E091E0BE0144E06A
:1036800050E00E947703009709F042C01092C005F5
:103690001092C1051092C2051092C305F801E25ABA
:1036A000FE4FD288C3E1D0E0EE24FF2487015F0102
:1036B0001FC0C801B7012AE030E040E050E00E949E
:1036C00054342D2D30E02053304079010027F7FC91
:1036D0000095102FE60EF71E081F191FC731D105E0
:1036E00011F4DD2405C0F501EC0FFD1FD0802196FB
:1036F0008D2D80538A3018F4C831D105D0F2E09274
:10370000C005F092C1050093C2051093C3050FC018
:103710008881803261F484E190E0A0E0B0E08093A1
:10372000C0059093C105A093C205B093C3058091D5
:10373000C0059091C105A091C205B091C305449701
:10374000A109B1098D569145A140B040E8F40E940D
:10375000DA2D2091C0053091C1054091C2055091EC
:10376000C305260F371F481F591F2093BC053093F0
:10377000BD054093BE055093BF0582E090E0909355
:10378000E9058093E80508C01092C0051092C105B4
:103790001092C2051092C3058091C0059091C10599
:1037A0000E947E0E9093F2058093F1050E94952E63
:1037B0006093C0057093C1058093C2059093C305C3
:1037C00078C08091F1059091F20589599E4F61E092
:1037D00070E008C08091F1059091F20589599E4FE3
:1037E00060E070E00E94DA0E5CC00E94CB0D59C010
:1037F00080E090E00E94E40B54C08091F10590912C
:10380000F20587599E4F0E9487174BC0C091F10562
:10381000D091F205BE0167597E4F82E091E044E00D
:1038200050E00E947703009739F5FE01E25AFE4FFF
:103830006785FE01E259FE4F40E150E020E030E0B4
:1038400011C0C901A3E0880F991FAA95E1F7220FC3
:10385000331F280F391F260F311D2053304061912F
:103860004F5F5F4F862F80538A3018F442315105E5
:1038700041F72031310510F020E030E0C9010E940D
:1038800014140FC086E090E09093E9058093E8055A
:103890000DC08091F1059091F20586599E4F0E94CE
:1038A000CE159093F2058093F10503C020E030E03F
:1038B00002C021E030E0C901DF91CF911F910F914B
:1038C000FF90EF90DF90BF90AF9008952F923F92BE
:1038D0004F925F926F927F928F929F92AF92BF9220
:1038E000CF92DF92EF92FF920F931F93CF93DF93CC
:1038F00076C48091E8059091E9058330910509F43B
:103900007CC18430910534F4009781F0029709F06E
:103910000AC24AC18530910509F4D8C185309105A4
:103920000CF4A6C1069709F0FEC113C180EF95E023
:1039300060EC72E04EE551E00E94942CAC0180EF07
:1039400095E06EE571E00E94992C9093F2058093CA
:10395000F105892B09F463C08091B4059091B505F8
:10396000892B89F188E591E00E9484078AE190E043
:103970001FC0E25AFE4F8AEB97E060814AE050E0B8
:103980000E944C338091FD059091FE054D9728F4DF
:103990008AEB97E060E071E004C08AEB97E068E2B0
:1039A00071E00E94EE338091FD059091FE05019635
:1039B0009093FE058093FD05E091FD05F091FE05D5
:1039C000EE31F105B0F28AE190E00E949B07892B6D
:1039D00009F4A9C10E94FB199093FC058093FB0593
:1039E000892B09F0A0C18091E8059091E905892B08
:1039F00009F099C180EF95E06EE571E040E050E09C
:103A000028EC30E00E943D2D9093F2058093F10563
:103A100081E090E09093FC058093FB0584C1809148
:103A20005C0190915D01039709F07DC12090D40560
:103A30003090D5054090D6055090D70520E4221649
:103A40002DE0320623E0420620E0520638F400E181
:103A5000A02E07E2B02EC12CD12C0CC0C201B101A6
:103A600024E130E040E050E00E949A34C901DA01DC
:103A70005C016D010E94952E2091CC053091CD0501
:103A80004091CE055091CF05621B730B840B950BB3
:103A9000A616B706C806D90608F045C10E94952E9D
:103AA0007B018C016090D0057090D1058090D2058B
:103AB0009090D305E618F70808091909C201B10169
:103AC0002CE030E040E050E00E949A342E153F0593
:103AD0004007510708F027C18091CC059091CD0592
:103AE000A091CE05B091CF0586159705A805B9051B
:103AF00049F10E94952E6093C0057093C105809393
:103B0000C2059093C30580EF95E00E948E2CAA0C0D
:103B1000BB1CCC1CDD1C8091D4059091D505A091D7
:103B2000D605B091D7058A199B09AC09BD098093C8
:103B3000540190935501A0935601B093570185E02D
:103B400090E056C082E090E090935D0180935C012C
:103B5000EAC00E94952E6093C4057093C5058093BA
:103B6000C6059093C7052091C0053091C1054091CD
:103B7000C2055091C305621B730B840B950B67390B
:103B800071058105910508F4CEC081E090E00E94A6
:103B9000DD0A9093F2058093F10581E090E0909327
:103BA000FC058093FB05BBC00E94952E2091C005AB
:103BB0003091C1054091C2055091C305621B730B42
:103BC000840B950B6A3F71058105910508F4ABC024
:103BD00081E090E00E94DD0A9093F2058093F10568
:103BE00081E090E09093FC058093FB0583E090E0FA
:103BF0009093E9058093E80596C00E94952E209148
:103C0000C0053091C1054091C2055091C305621BAA
:103C1000730B840B950B645F71408040904008F4F7
:103C200082C080EF95E00E948E2C80915C01909183
:103C30005D01892B31F082E090E090935D018093EB
:103C40005C0184E090E09093E9058093E80580E0D2
:103C500090E00E9489108091B4059091B5051816E6
:103C600019060CF060C088E491E00E9484075BC0F4
:103C70000E94DA2D2091BC053091BD054091BE0512
:103C80005091BF05261737074807590708F04BC062
:103C900081E090E00E94891080EF95E00E94912CD5
:103CA0000E94952E6093D0057093D1058093D20524
:103CB0009093D3058091B4059091B5051816190617
:103CC00074F589E391E00E94840729C00E94952E33
:103CD0002091C0053091C1054091C2055091C305A6
:103CE000621B730B840B950B20915401309155018D
:103CF0004091560150915701621773078407950749
:103D000090F080EF95E00E94912C0E94952E609398
:103D1000D0057093D1058093D2059093D30510926E
:103D2000E9051092E8050E94952E209158013091E6
:103D3000590140915A0150915B01621B730B840B36
:103D4000950B615375478040904030F18091E805B4
:103D50009091E905069701F180EA60E00E94CC0F9E
:103D60001092B1051092B0050E94952E20E335E720
:103D700040E050E00E949A34CA01B90120E335E7DF
:103D800040E050E00E945434609358017093590110
:103D900080935A0190935B018091FB059091FC0503
:103DA000019709F045C10E94952E2091CC053091D4
:103DB000CD054091CE055091CF05621B730B840B4E
:103DC000950B615177428040904030F1C0EED5E0D4
:103DD00009C088819981AA81BB818C839D83AE8330
:103DE000BF83249785E0C43DD80799F71092FE055C
:103DF0001092FD050E94952E2091CC053091CD05A5
:103E00004091CE055091CF05621B730B840B950B2F
:103E10006C837D838E839F830E94952E6093CC0557
:103E20007093CD058093CE059093CF0580915C0172
:103E300090915D0102970CF4DEC06090D8057090FF
:103E4000D9058090DA059090DB0561147104810436
:103E5000910409F4D0C02090DC053090DD0540903D
:103E6000DE055090DF05211431044104510409F4AA
:103E7000C2C02091E0053091E1054091E2055091EA
:103E8000E305211531054105510509F4B4C08091C0
:103E9000E4059091E505A091E605B091E70500974E
:103EA000A105B10509F4A7C082017101E60CF71C58
:103EB000081D191DE20EF31E041F151FE80EF91E42
:103EC0000A1F1B1FB2E016950795F794E794BA9561
:103ED000D1F7E092D405F092D5050093D605109362
:103EE000D705D801C701805C944DA140B0408154F2
:103EF0009840AC46B04008F07CC0C801B70124E14E
:103F000030E040E050E00E949A34C901DA015701E4
:103F10006801A81AB90ACA0ADB0A6A147B048C046D
:103F20009D0408F466C09C01AD012E0D3F1D401F8D
:103F3000511F261537054805590508F45AC02A149B
:103F40003B044C045D0408F454C0221533054405B9
:103F5000550508F44EC0E090E005F090E1050091B1
:103F6000E2051091E305EA14FB040C051D0508F4B5
:103F700040C02E153F0540075107D8F1E090E405F9
:103F8000F090E5050091E6051091E705EA14FB04C1
:103F90000C051D0570F12E153F054007510748F12E
:103FA00080915C0190915D01029729F583E090E09A
:103FB00090935D0180935C018091B4059091B5056B
:103FC000892BC9F08FE291E00E9484074091D405CB
:103FD0005091D5056091D6057091D7058AEB97E091
:103FE0002AE030E00E943D338AE291E00E9484079B
:103FF00002C00E94B9084091F1055091F20580EF8E
:1040000095E06EE571E00E94322DEEE5F1E080E092
:1040100090E002C01192019622E0803C9207D0F31A
:104020009093FE058093FD051092FC051092FB0510
:104030000E94340990935D0180935C0182E00E94AC
:10404000F62F9093FE058093FD054091F705509162
:10405000F8056091F9057091FA050097D9F44115BA
:1040600051056105710559F40E94952E6093F7057D
:104070007093F8058093F9059093FA05A9C00E9402
:10408000952E6093F3057093F4058093F505909356
:10409000F6059EC0411551056105710509F459C029
:1040A0008091F3059091F405A091F505B091F60586
:1040B0000097A105B10509F44CC08E5E9240A04066
:1040C000B040841B950BA60BB70B835E9440A040B9
:1040D000B04008F03EC060E070E08091B60590917D
:1040E000B705892B11F461E070E07093B705609318
:1040F000B60589E00E94A22F8091B6059091B70580
:104100002091EE053091EF05019789F4232B21F4DE
:104110008DE191E00E94840787E090E09093E905AB
:104120008093E80580EF95E00E948E2C12C0232B2F
:1041300021F484E191E00E94840781E090E00E94F4
:10414000891080EF95E00E94912C1092E905109261
:10415000E8051092F3051092F4051092F5051092FF
:10416000F6051092F7051092F8051092F9051092D5
:10417000FA052EC06091B0057091B105625E7B4F6B
:104180008AEB97E041E050E00E943034019749F417
:104190008091B0059091B10501969093B1058093FF
:1041A000B0058091B0059091B105849731F480916C
:1041B00041048F3711F40E9471058091B0059091F0
:1041C000B1058036910524F01092B1051092B0052A
:1041D0008AEB97E00E945A31181619065CF280911A
:1041E000EA059091EB05892B09F083CBDF91CF9104
:1041F0001F910F91FF90EF90DF90CF90BF90AF9005
:104200009F908F907F906F905F904F903F902F90F6
:104210000895EF92FF920F931F938091E3068530EC
:1042200011F5E090E806F090E9060091EA06109199
:10423000EB068091E4069091E506A091E606B09128
:10424000E706E80EF91E0A1F1B1F0E94952EAA27DB
:1042500097FDA095BA2F8E159F05A007B10718F0FE
:1042600086E08093E3068091E3061F910F91FF9013
:10427000EF90089585E08093E3060E94952EAA278B
:1042800097FDA095BA2F8093E4069093E506A0933E
:10429000E606B093E7060E94B72482E00895FF92F5
:1042A0000F931F93CF93DF938C01F62E1092EC06A1
:1042B0001092ED068091EE068F5F8093EE0680E906
:1042C00091E0D801FC011D923197E9F76091EE066B
:1042D00070E0706E4091DE075091DF07C80124E462
:1042E00030E00E940B28D80116962091EF063091FD
:1042F000F006C901FC0186E001900D928150E1F7C2
:10430000C8016FEF70E046E050E00E94700382E861
:10431000D80151968C93519781E157968C938FEFEA
:104320009FEFAFEFBFEFF801868F978FA0A3B1A3E8
:1043300083E485A312A284E483A3BA9681E0D80122
:104340009A968C93818386E0828313828091DD0626
:104350009091DE06A091DF06B091E00684839583FC
:10436000A683B7838091E1069091E20691878087CA
:10437000D801DA961D921D921D921C92DD977C96B3
:104380002091EF063091F006C901DC0186E00D9026
:1043900001928150E1F7D801AA5EBE4F93E6FD017C
:1043A000919382E811968C93DF01119683E58183C6
:1043B000FD01319611969C93DF01119685E381836F
:1043C000FD01319691E011969C93DF011196F182E7
:1043D0009D012F5F3F4F8DE311968C93F90131962C
:1043E00087E0D90111968C939183EF012296409139
:1043F000EF065091F00620E030E0FE01E20FF31FDF
:10440000DA01A20FB31F8C9180832F5F3F4F2630BC
:10441000310599F78CE08E838AE08F83289620E01F
:1044200030E0FE01E20FF31FD901A258BA4F8C9180
:1044300080832F5F3F4F2A30310599F72A96D0931A
:10444000F206C093F1062A97B3E0FB1609F042C0CA
:1044500082E38A8794E09B87E091DE07F091DF0793
:1044600080818C87E091DE07F091DF0781818D8765
:10447000E091DE07F091DF0782818E87E091DE0711
:10448000F091DF0783818F8786E3888B998B629613
:10449000D093F206C093F1066297E091E007F091A5
:1044A000E10780818A8BE091E007F091E10781814B
:1044B0008B8BE091E007F091E10782818C8BE0919A
:1044C000E007F091E10783818D8B6696D093F20629
:1044D000C093F106A091F106B091F206FD0187E3C9
:1044E000819393E011969C93DF01119681E0818383
:1044F0009D012F5F3F4F11969C93F901319686E005
:10450000D90111968C938FEF81833296F093F20646
:10451000E093F106E01BF10BBA97C801BF010E94BE
:104520006929DF91CF911F910F91FF90089563E06A
:1045300070E00E944F2183E08093E3060895DF92AC
:10454000EF92FF920F931F93CF93DF938C017B0128
:10455000E091DE07F091DF07EC018AAD9BADACADD9
:10456000BDAD80839183A283B383F801E65EFE4FE5
:10457000E00EF11EDF011196D180ED0121968081C0
:104580008630C1F0873030F4813051F0833009F04B
:1045900057C00BC0833399F0863309F051C042C035
:1045A000E091E407F091E50741C0E091E207F09166
:1045B000E3073CC0E091DC07F091DD0737C01196BE
:1045C0006C9170E080E090E0982F872F762F66271F
:1045D0002981620F711D811D911D982F872F762FC4
:1045E00066272A81620F711D811D911D982F872FCB
:1045F000762F66272B81620F711D811D911D982FCB
:10460000872F762F662728EE33E040E050E00E94A7
:1046100054346093E8067093E9068093EA06909319
:10462000EB060EC0E091E007F091E10711968D9145
:104630009D910D90BC91A02D80839183A283B38323
:10464000FE01ED0DF11DEE15FF0508F493CFC80135
:104650000E94972281E0DF91CF911F910F91FF90EF
:10466000EF90DF900895FC0166347105A0F183A1FD
:10467000833489F5DF019A9682A5823061F514961C
:104680002D913D914D915C9117978091DD06909110
:10469000DE06A091DF06B091E006281739074A0729
:1046A0005B07C9F4E65EFE4F8081EA51F140853335
:1046B00091F4E45EFE4F8081EC51F140823019F0BC
:1046C000853049F404C0CF010E949F220895CF0194
:1046D0000E943A21089580E00895CF92DF92EF92F0
:1046E000FF920F931F93CF93DF93EC017093F0062B
:1046F0006093EF065093DF074093DE073093E507A2
:104700002093E4071093E3070093E207F092E10798
:10471000E092E007D092DD07C092DC0780E090E0F5
:104720000E94412F0E944E030E944903AA2797FD31
:10473000A095BA2F8F5D9C4BAA49BF4F8093DD0691
:104740009093DE06A093DF06B093E0061092E20697
:104750001092E10680E090E0E091DE07F091DF0743
:10476000E80FF91F1082E091E407F091E507E80FE8
:10477000F91F1082E091E207F091E307E80FF91FBB
:104780001082E091E007F091E107E80FF91F108235
:10479000E091DC07F091DD07E80FF91F1082019628
:1047A00084309105C9F6E091EF06F091F00685811D
:1047B00082958F708F5B8093860585818F708F5B6C
:1047C000809387050E94C024CE0161E070E00E94C2
:1047D0004F2181E08093E306DF91CF911F910F91EC
:1047E000FF90EF90DF90CF9008958AE061E00E9403
:1047F000632F8AE061E00E94A22F8BE061E00E94BB
:10480000632F8DE061E00E94632F8CE060E00E94E6
:10481000632F8BE061E00E94A22F8BE060E00E949A
:10482000A22F8DE060E00E94A22F81E58CBD8DB5A6
:1048300081608DBD08950F931F93CF93DF938C01FB
:10484000EB01F8948091890560E00E94A22F8AE72D
:104850008EBD0DB407FEFDCF08C088818EBD0DB49E
:1048600007FEFDCF21960150104001151105A9F753
:104870008091890561E00E94A22F7894DF91CF9109
:104880001F910F9108950F931F93CF93DF93EC0126
:104890008B01F8948091890560E00E94A22F8AE341
:1048A0008EBD0DB407FEFDCF09C01EBC0DB407FEC2
:1048B000FDCF8EB5F80181938F0121972097A9F73D
:1048C0008091890561E00E94A22F7894DF91CF91B9
:1048D0001F910F910895FF920F931F93082F162F8A
:1048E000F42EF8948091890560E00E94A22F1F7138
:1048F000102B1EBD0DB407FEFDCFFEBC0DB407FE90
:10490000FDCF8091890561E00E94A22F78941F91CC
:104910000F91FF9008951F93182F282F30E02076D5
:1049200030708091F30690E02817390781F080EA13
:104930006FE143E00E946B24412F40764093F306E1
:1049400042954695477080E86FE10E946B241F9165
:1049500008950F931F93182F062F0E948B2480E435
:10496000612F402F0E946B241F910F910895609139
:10497000F6066E7F6093F60688E30E94A9240895E8
:104980006091F60661606093F60688E30E94A924B0
:104990000895682F677085E70E94A92408950F93F2
:1049A0001F93182F072F0E94A924812F8F5F602F3C
:1049B0000E94A9241F910F9108950F931F93182F00
:1049C000062FF8948091890560E00E94A22F802F25
:1049D0008F71812B8EBD0DB407FEFDCF1EBC0DB4B3
:1049E00007FEFDCF07FF04C01EBC0DB407FEFDCFC0
:1049F0001EB58091890561E00E94A22F7894812FD5
:104A00001F910F9108951F93182F0E948B2480E00F
:104A1000612F0E94DD241F910895AF92BF92CF9223
:104A2000DF92EF92FF920F931F93DF93CF9300D00B
:104A3000CDB7DEB76C015B0189E30E9403258823B3
:104A400019F400E010E051C06091F4067091F50691
:104A500080E00E94CF2482E090E08E010F5F1F4F24
:104A6000B8010E94432489819A819093F50680932E
:104A7000F40682E090E0B8010E944324E980FA80C5
:104A800082E090E0B8010E944324898187FD03C041
:104A900000E010E00DC0C7010497860101501040EE
:104AA0008017910708F48C01C801B5010E944324C6
:104AB0006091F4067091F5068CE00E94CF2460911D
:104AC000F4067091F5066150704089E16F3F7807F8
:104AD00020F08CE06EEF79E101C08CE00E94CF24E1
:104AE00080E86EE140E40E946B24C8010F900F90B3
:104AF000CF91DF911F910F91FF90EF90DF90CF90BA
:104B0000BF90AF90089582E70E940325863008F099
:104B10008F5F089580EA6EE140E20E946B248DE190
:104B20000E9403258823D9F380E86FE144E00E94C6
:104B30006B24089580EA6FE144E00E946B248DE1CC
:104B40000E94032582FDFBCF8FE10E94032583FD98
:104B5000FBCF80E86EE148E00E946B2480E86EE1C4
:104B600040E20E946B2408950F931F93CF93DF932D
:104B7000EC018B010FC08CE10E94032581FF0AC06C
:104B800080E86FE140E80E946B2480EA6FE140E832
:104B90000E946B2480E06FE10E94DD2483FDEBCF57
:104BA00082E06FEF79E10E94CF24BE016150764E22
:104BB00086E00E94CF248AE760E040E00E946B24F8
:104BC000CE01B8010E941B2480E86FE148E00E94FA
:104BD0006B24DF91CF911F910F9108950F931F9335
:104BE000982F162F072F84ED692F0E94A92486ED98
:104BF000612F0E94A92487ED602F0E94A92404C080
:104C00008FE090E00E94FC2E8AEE0E94032580FD3A
:104C1000F7CF1F910F9108950F931F938C01862F4B
:104C20006093890561E00E94632F8091890561E0AE
:104C30000E94A22F78948FEF60E04FEF0E946B24C8
:104C400062E370E080E090E00E94A32E1092F506EF
:104C50001092F40688E060E070E00E94CF248CE0BF
:104C600060E070E00E94CF248AE06EEF79E10E945C
:104C7000CF2484E06FEF79E10E94CF2486E06FEFCC
:104C80007FE10E94CF2481EB8093F60688E361EBFD
:104C90000E94A92488E26FE370E30E94CF2480E39E
:104CA00069EF77EF0E94CF2480EC6DE00E94A92489
:104CB00081EC60E00E94A92480E862EC42E30E945B
:104CC0006B2486EC62E17CE00E94CF2484EC62E1FC
:104CD0000E94A9248AEC6CED75E00E94CF2484EE3A
:104CE000F80160810E94A92485EEF80161810E948B
:104CF000A92482EEF80162810E94A92483EEF801C2
:104D000063810E94A92480EEF80164810E94A92495
:104D100081EEF80165810E94A92480E160E071E0E4
:104D20000E94EE258FE10E948B2480E86BE140EC2D
:104D30000E946B2480E86FE144E00E946B241F9185
:104D40000F910895682F84ED0E94A92482ED61E0FF
:104D50000E94A9248FE090E00E94FC2E8AEE0E941F
:104D6000032580FDFBCF82ED60E00E94A92489ED40
:104D70000E94032590E0089581E10E94A22620E090
:104D8000892B09F021E0822F0895CF92DF92EF92D4
:104D9000FF920F931F93CF93DF936C01413081F407
:104DA000685070407B0100E010E0685F7F4F21E1B8
:104DB00030E040E050E0E20EF31E041F151F15C066
:104DC000423021F0EE24FF2487010FC0685070406C
:104DD0007B0100E010E0685F7F4F86E090E0A0E09C
:104DE000B0E0E80EF91E0A1F1B1FF601EB0116C00A
:104DF000808190E0A0E0B0E0BA2FA92F982F8827FB
:104E0000218130E040E050E0822B932BA42BB52B86
:104E1000E80EF91E0A1F1B1F32962297C230D105D9
:104E200038F7FB01EE7FEC0DFD1D60FF15C08081A2
:104E300090E0A0E0B0E0BA2FA92F982F882708C0F3
:104E40002FEF3FEF40E050E0E222F322042315234E
:104E5000E80EF91E0A1F1B1FC801AA27BB270097CF
:104E6000A105B10569F7970120953095C901DF913A
:104E7000CF911F910F91FF90EF90DF90CF90089509
:104E8000CF93DF93EC015093FD0640938E0520E015
:104E900030E0F901EC5EF84FDB01A20FB31F8C91FB
:104EA00080832F5F3F4F2430310599F720E030E0B9
:104EB000F901EA51F84FDE01A20FB31F8C918083F4
:104EC0002F5F3F4F2630310599F7DF91CF9108953D
:104ED000FC0169327105B0F08485883099F48585CC
:104EE000863081F4DF019696E4E1F7E09C918081C1
:104EF000981741F41196319687E0E831F807B1F739
:104F000081E0089580E00895FC016A327105D0F0D7
:104F100084858830B9F485858823A1F48685853415
:104F200089F4DF01E4E1F7E05E969C915E97808171
:104F3000981741F41196319687E0E831F807A1F708
:104F400081E0089580E008950F931F938C01FC0188
:104F5000108E118E80E4848B158A868BC8010E9684
:104F600064E170E040E00E94C526F801908F818FD7
:104F70001F910F910895AC01FC01A4E1B7E0828D6F
:104F8000868F8D91828F319687E0A831B807B9F767
:104F9000CA010E94A4270895FC01B99694E080817B
:104FA000680F711D84816483442311F0808301C0E4
:104FB000108291503197992319F0672F7727EFCFFF
:104FC00008950F931F938C01FC0194A182A184A3E7
:104FD00092A395A183A185A393A3C8010E94CC2786
:104FE000F80112AA13AA80E586A71F910F910895D0
:104FF0006A5C7F4FDC01A60FB71F6653704003C089
:105000008D936F5F7F4FFA014F5F5F4F84918823CD
:10501000B9F7CB010895FF920F931F93CF93DF93BE
:10502000EC01F62E072FBA01122F932FAE019E012D
:10503000A0E0B0E0FD01E65FF84F8081F9018083D8
:10504000FD01EA51F84F8081F901868311962F5FA7
:105050003F4FA630B10571F788E08C871D86DE01D1
:10506000E1E3F4E084911E968C931E97319611969D
:1050700084E0EA33F807B1F7188A81E18F8BA0E06A
:10508000B0E0FB01EA0FFB1F8081FA01868FFD0172
:10509000EC5EF84F8081FA01828F11964F5F5F4F6F
:1050A000A430B10571F79CA31DA30AA3FBA21EA205
:1050B00018A619A6DF91CF911F910F91FF90089527
:1050C000AC0181E080938A0520E030E0F901EA5FDD
:1050D000F84FDA01A20FB31F8C9180832F5F3F4FEF
:1050E0002430310599F70895CF93DF93EB01BA018E
:1050F000DA010D900020E9F71197A41BB50BE69695
:10510000AC014C0F5D1FE6979D0108C0FB0181912A
:10511000BF01FA018193AF012150304021153105C3
:10512000A9F79E012A0F3B1FC901DF91CF91089576
:10513000FF920F931F93CF93DF93EC01F62E142F62
:10514000022FAC01DC0120E030E0F901E65FF84F0E
:1051500080818C93F901EA51F84F808116968C93E7
:1051600016972F5F3F4F11962630310571F788E073
:105170008C871D86DE01E1E3F4E084911E968C931A
:105180001E973196119684E0EA33F807B1F78CE266
:10519000898B86E08F8B20E030E0F901E05FF84FEB
:1051A0008081FA01868FF901EC5EF84F8081FA0167
:1051B000828F2F5F3F4F4F5F5F4F2430310569F77C
:1051C000CE010E94A4271CA30DA38BE08AA3FBA2FF
:1051D000FE01B69680E011928F5F8830E1F78091F2
:1051E0008F0588A78D5F80938F0580E68EA782E06C
:1051F0008FA794E098AB19AA1AAA1BAA1CAA1DAAE9
:105200008EAB9FAB88AF86E289AFCE014A9660E253
:1052100070E042E00E94C5269AAB8BAB8AE390E037
:10522000BE010E94B425DF91CF911F910F91FF9095
:105230000895CF93DF93EC01AC0126EE37E0FC013B
:10524000D9019FEF90838D918683319687E0AC3EA4
:10525000B807C1F788E08C8786E08D87DE01E9E238
:10526000F4E084911E968C931E973196119684E0FB
:10527000E133F807B1F7F90181919F01FA01868BBB
:1052800010A24F5F5F4FF7E02C3E3F07A1F7DE0112
:105290005C9620E030E0FB01E20FF31F80811A965C
:1052A0008C931A97F901EC5EF84F80818D932F5FF4
:1052B0003F4F2430310579F780918A0588608093CB
:1052C0008A058AE290E0BE010E94B425DF91CF9169
:1052D0000895DF92EF92FF920F931F938C017B0151
:1052E0008CE190E0E80EF91EF801F08A84EE9FEF61
:1052F000E80EF91EDE2C9CE1D90ED18AC8010E946D
:10530000A427E8E0F0E0EE0EFF1EF801F6A2FCEEA6
:10531000DF0EF801D7A288E090E0E80EF91EC80180
:105320004A96B70141E00E94C526F80190A781A7DF
:10533000C7014A96B8010E94B4251F910F91FF90B2
:10534000EF90DF900895EF92FF920F931F938C01DF
:105350007B01CB018896F801908B818BC8010E945C
:10536000A427F80112AA13AA8CE190E0E80EF91E16
:10537000C8014A96B70142E00E94C526F80192ABE7
:1053800083ABC7014A96B8010E94B4251F910F91C3
:10539000FF90EF900895CF93DF93EC01FC01A6EE10
:1053A000B7E0868180838D918683319687E0AC3E1D
:1053B000B807B9F7842F80618FA7443029F06115B1
:1053C000710511F461E070E0CE0141E00E94E12737
:1053D000188A88E2898BCE010E94BB2784E088ABC3
:1053E00019AACE014A966CE170E042E00E94C526FF
:1053F0009AAB8BAB86E390E0BE010E94B425DF91AF
:10540000CF910895EF92FF920F931F938C017B0130
:105410006091FE067091FF0640E00E94CB2989E171
:10542000F80187A7C801B7010E94A3291F910F9116
:10543000FF90EF900895CF93DF93EC01FC01A6EE6F
:10544000B7E0868180838D918683319687E0AC3E7C
:10545000B807B9F7188A8CE2898BCE010E94BB2766
:1054600082E18FA7CE0161E070E040E00E94E12779
:105470001EA21FA280918F0588A719A68D5F809319
:105480008F0582E08EAB84E08FAB95E098AF19AECC
:1054900080E68EA798AB88E789ABCE014A9660E29A
:1054A00070E042E00E94C5269AAB8BAB8AE390E0A5
:1054B000BE010E94B425DF91CF9108950F931F93F1
:1054C000CF93DF93EC018B01FC01A6EEB7E0868160
:1054D00080838D918683319687E0AC3EB807B9F71B
:1054E000CE010E94BB271AA28CA1883F18F08DA183
:1054F0008F5F8DA38CA1885F8CA3C801BE010E9421
:10550000B425DF91CF911F910F910895CF93DF9331
:10551000AC01EC0126EE37E0FC01D90186818083E5
:105520008D918683319687E0AC3EB807B9F7FA01D2
:10553000148A82E0858B8E8988A3F90181919F016D
:105540008E8B2196F7E02C3E3F07A9F7FA017C9657
:10555000A4E1B7E0808182878D91819387E0A831B3
:10556000B807C1F78AE290E0BA010E94B425DF9142
:10557000CF910895EF92FF920F931F93CF93DF93F4
:10558000EC017B016115710509F040C080918A052D
:1055900080FD04C080918A0582FF0FC080918B0539
:1055A00090918C05892B49F40E94BC26882329F010
:1055B000CE0166E077E00E94192980918B059091D9
:1055C0008C05019690938C0580938B058091F7064E
:1055D000813009F08FC180918A0581FF8BC182E003
:1055E0008093F70680918D058F5F80938D058F7175
:1055F0006091F8066295660F607E682BCE0140913F
:10560000F9062091FA060E94982874C10E94682722
:10561000882341F18D89813019F4CE010E94862AB8
:1056200080918A0583FF66C18D89823009F062C14D
:10563000E6E0F7E0DE015C969C915C97808198172C
:1056400009F058C11196319687E0EA30F80799F7CA
:10565000EAE0F7E08E898193219697E0E031F9073F
:10566000C9F752C1CE01B7010E948427882309F4EB
:1056700041C19F89913149F48AA18823C9F48BA142
:105680008533B1F46AE270E037C1913089F48AA1C0
:10569000883071F4E0910407F0910507309719F014
:1056A000CE014A960995CE01B7010E945E2A22C119
:1056B00086E3E816F10418F4963009F01BC19CA1AA
:1056C0009B3009F0C9C0D093FC06C093FB06DE01F5
:1056D000E0E1F7E05A969C915A978081981709F07B
:1056E00009C11196319697E0E431F90799F710C195
:1056F000E0910007F0910107309709F4A3C08DA154
:1057000082958695877063E040E050E020E030E0CD
:10571000099598C0988980E02989022F10E0082B0C
:10572000192B8EA582958F70482F50E0CA01880FE3
:10573000991F880F991F081B190B0451104017FF60
:1057400002C000E010E0B8018091F706823089F5D0
:1057500031FF20C034FF1EC0CE0160E070E040E0A9
:105760000E94CB2988E18FA7E0910207F0910307FF
:10577000309719F460E070E006C08BA182958695A1
:1057800087700995BC0183E08093F706CE010E94E3
:10579000A329B0C081E08093F7068FA584FF03C0E2
:1057A00060E070E003C0B8016F5F7F4FCE0144E05E
:1057B0008CC0843039F4E0910007F09101073097F4
:1057C00089F432C0833099F584E08093F706E09144
:1057D0000007F0910107309739F18EA582958F70FF
:1057E000482F50E0440F551F440F551FC70108971D
:1057F0004E5D5F4F8417950708F4AC01C801840F14
:10580000951FE816F90610F0980103C09701241BB4
:10581000350B8DA182958695877060E00995882368
:1058200019F0CE01B8010BC0CE01B8014DC08530D2
:1058300009F460C030FF0AC06F5F7F4FCE0149E0BE
:105840000E94CB2985E08093F70654C0011511050D
:1058500009F452C0CE0138C08091FD06981709F0B6
:1058600049C09DA180918E05981709F043C08FA56E
:1058700081FF04C0CE010E941B2A3CC084FF3AC0B5
:10588000988980E02989422F50E0482B592B2EA57A
:10589000822F82958F7090E0880F991F880F991F33
:1058A000481B590B4451504057FF02C040E050E0A4
:1058B0005093FF064093FE06452B51F48FA580FFC1
:1058C00019C0CE0160E070E040E00E94CB2912C018
:1058D0008EA582958F70682F70E0660F771F660F18
:1058E000771F6E5D7F4F88EF9FEFE80EF91EE6167B
:1058F000F70610F460E070E0CB01DF91CF911F91CB
:105900000F91FF90EF90089582E080938A05F2CF87
:105910008FA5382F82FDECCEFDCE08950E949A25EA
:1059200008950E948A250895CB01BA010E940D2591
:105930000895CB01BA010E94BA2A08952F923F928E
:105940005F926F927F928F929F92AF92BF92CF920F
:10595000DF92EF92FF920F931F93DF93CF93CDB718
:10596000DEB72A970FB6F894DEBF0FBECDBF3B015E
:105970005A8349833C832B83FE82ED82D886CF8273
:10598000BA86A98614010E94952EAC01CB01DA01DA
:105990004C015D01C3016B817C814D815E812F8152
:1059A000388509851A857101CE8CDF8C0E946D23A4
:1059B00088E0582E89819A81B3010E940D258C01BF
:1059C000C301B8010E94BA2A892BA1F7C301B8010B
:1059D0000E9433230E940921853011F481E026C002
:1059E0000E94952EA50194012059384E4F4F5F4FCC
:1059F0002617370748075907E8F60E94952E5A944C
:105A0000A1F0AC01CB01DA014C015D01C3016B8156
:105A10007C814D815E812F81388509851A857101D0
:105A2000CE8CDF8C0E946D23C5CF80E02A960FB606
:105A3000F894DEBF0FBECDBFCF91DF911F910F91C4
:105A4000FF90EF90DF90CF90BF90AF909F908F909E
:105A50007F906F905F903F902F900895CB010E94B0
:105A600060280895CB01BA010E94022A0895CB0153
:105A7000BA01A9010E9474280895CB01BA01A901B5
:105A80000E94F8270895CB01BA01A9010E9440277E
:105A900008950E9483250895CF93DF93CB01642F4F
:105AA0000E940C2682E00E94C9246AE070E080E037
:105AB00090E00E94A32EC0E0D0E084E160E878E3AB
:105AC0000E94EE2564EF71E080E090E00E94A32E3A
:105AD00084E160E979E30E94EE2564EF71E080E003
:105AE00090E00E94A32E2196C330D10531F784E1C6
:105AF00066E774E30E94EE2564E670E080E090E0E3
:105B00000E94A32EDF91CF9108954AE00E944C2D70
:105B100008950E94F5230895F999FECF72BD61BDE5
:105B2000F89A80B50895F999FECF1FBA72BD61BD8C
:105B300040BD0FB6F894FA9AF99A0FBE0895809175
:105B40002307909124070895609390057093910521
:105B50008093920590939305089560931B0770932B
:105B60001C0780931D0790931E072091900530918C
:105B700091054091920550919305260F371F481FBC
:105B8000591F20931F0730932007409321075093FC
:105B9000220782E090E090932407809323070E94DD
:105BA000952E60932507709326078093270790937F
:105BB00028070895EF92FF920F931F931CC02F5F49
:105BC0003F4F4F4F5F4F20931B0730931C0740936D
:105BD0001D0750931E0788EE93E0A0E0B0E0E80EAA
:105BE000F91E0A1F1B1FE0922507F092260700935B
:105BF0002707109328070E94952EE0902507F09024
:105C0000260700912707109128076E197F09800B3E
:105C1000910B20911B0730911C0740911D0750915B
:105C20001E07685E73408040904048F680911F07D1
:105C300090912007A0912107B091220728173907DA
:105C40004A075B07E8F0E0911907F0911A073097CF
:105C500049F00995611571058105910519F00E94BA
:105C6000AD2D0EC020E030E08091230790912407F5
:105C7000892B11F021E030E0309324072093230793
:105C800060911B0770911C0780911D0790911E0762
:105C90001F910F91FF90EF9008951F920F920FB6F2
:105CA0000F9211242F933F938F939F93AF93BF93A2
:105CB00080912D0790912E07A0912F07B09130076A
:105CC000309131070196A11DB11D232F2D5F2D3776
:105CD00020F02D570196A11DB11D2093310780930F
:105CE0002D0790932E07A0932F07B0933007809134
:105CF000290790912A07A0912B07B0912C070196B4
:105D0000A11DB11D8093290790932A07A0932B070B
:105D1000B0932C07BF91AF919F918F913F912F919D
:105D20000F900FBE0F901F9018958FB7F894209189
:105D30002D0730912E0740912F07509130078FBFCC
:105D4000B901CA0108959B01AC017FB7F894809115
:105D5000290790912A07A0912B07B0912C0766B5CF
:105D6000A89B05C06F3F19F00196A11DB11D7FBF13
:105D7000BA2FA92F982F8827860F911DA11DB11D1D
:105D800062E0880F991FAA1FBB1F6A95D1F7BC015B
:105D90002DC0FFB7F8948091290790912A07A09110
:105DA0002B07B0912C07E6B5A89B05C0EF3F19F073
:105DB0000196A11DB11DFFBFBA2FA92F982F8827CB
:105DC0008E0F911DA11DB11DE2E0880F991FAA1F22
:105DD000BB1FEA95D1F7861B970B885E9340C8F2EC
:105DE000215030404040504068517C4F21153105D2
:105DF0004105510571F60895019739F0880F991FF3
:105E0000880F991F02970197F1F70895789484B548
:105E1000826084BD84B5816084BD85B5826085BDA6
:105E200085B5816085BDEEE6F0E08081816080838C
:105E3000E1E8F0E01082808182608083808181606F
:105E40008083E0E8F0E0808181608083E1EBF0E036
:105E5000808184608083E0EBF0E0808181608083DA
:105E6000EAE7F0E0808184608083808182608083C3
:105E70008081816080838081806880831092C100EE
:105E80000895982F8E3008F09E5097708091940559
:105E90008295880F880F807C892B80937C0080916D
:105EA0007A00806480937A0080917A0086FDFCCF2E
:105EB0002091780040917900942F80E030E0282BE9
:105EC000392BC9010895CF93DF93482F50E0CA01C1
:105ED00081599A4FFC013491455A5A4FFA018491E5
:105EE000882369F190E0880F991FFC01E35CFA4F69
:105EF000A591B491FC01E95BFA4FC591D491662359
:105F000051F42FB7F8948C91932F909589238C930B
:105F1000888189230BC0623061F42FB7F8948C918B
:105F2000932F909589238C938881832B88832FBF0F
:105F300006C09FB7F8948C91832B8C939FBFDF9101
:105F4000CF910895482F50E0CA018D579A4FFC0118
:105F50002491CA0181599A4FFC019491455A5A4F94
:105F6000FA013491332309F440C0222351F1233044
:105F700071F0243028F42130A1F0223011F514C042
:105F80002630B1F02730C1F02430D9F404C080911C
:105F900080008F7703C0809180008F7D8093800088
:105FA00010C084B58F7702C084B58F7D84BD09C0D1
:105FB0008091B0008F7703C08091B0008F7D809377
:105FC000B000E32FF0E0EE0FFF1FE95BFA4FA59161
:105FD000B4912FB7F894662321F48C91909589237E
:105FE00002C08C91892B8C932FBF0895682F70E08D
:105FF000CB018D579A4FFC012491CB0181599A4FC7
:10600000FC014491655A7A4FFB019491992319F44C
:1060100020E030E03CC0222351F1233071F02430E5
:1060200028F42130A1F0223011F514C02630B1F04F
:106030002730C1F02430D9F404C0809180008F77DC
:1060400003C0809180008F7D8093800010C084B554
:106050008F7702C084B58F7D84BD09C08091B00068
:106060008F7703C08091B0008F7D8093B000892F1F
:1060700090E0880F991F8F5A9A4FFC01A591B49117
:106080008C9120E030E0842311F021E030E0C90160
:10609000089508951F920F920FB60F9211242F9317
:1060A0003F934F938F939F93EF93FF938091C00003
:1060B00082FD1DC04091C600209172073091730788
:1060C0002F5F3F4F2F733070809174079091750749
:1060D0002817390771F0E0917207F0917307EE5CB1
:1060E000F84F4083309373072093720702C080916A
:1060F000C600FF91EF919F918F914F913F912F910A
:106100000F900FBE0F901F901895E091C607F09169
:10611000C707E05CFF4F8191919120813181821B03
:10612000930B8F739070892B11F00E944930089562
:106130001F920F920FB60F9211242F933F938F93BC
:106140009F93EF93FF932091B6073091B70780910B
:10615000B8079091B9072817390731F48091C10029
:106160008F7D8093C10014C0E091B807F091B9070A
:10617000EA58F84F20818091B8079091B9070196AD
:106180008F7390709093B9078093B8072093C600DF
:10619000FF91EF919F918F913F912F910F900FBEA3
:1061A0000F901F901895AF92BF92DF92EF92FF92DF
:1061B0000F931F93CF93DF93EC017A018B01DD24C2
:1061C000403081EE580780E0680780E0780711F0E2
:1061D000DD24D39491E0A92EB12CEC89FD89DD203A
:1061E00069F0C50108A002C0880F991F0A94E2F760
:1061F000808360E079E08DE390E005C0108260E884
:1062000074E88EE190E0A80197010E949A34215031
:10621000304040405040569547953795279580E14E
:106220002030380720F0DD2011F0DD24D6CFE889BA
:10623000F9893083EA89FB89208319A2EE89FF89D5
:10624000408121E030E0C9010C8C02C0880F991F09
:106250000A94E2F7482B4083EE89FF894081C90107
:106260000D8C02C0880F991F0A94E2F7482B4083D7
:10627000EE89FF894081C9010E8C02C0880F991FE9
:106280000A94E2F7482B4083EE89FF8980810F8CC6
:1062900002C0220F331F0A94E2F72095282320839F
:1062A000DF91CF911F910F91FF90EF90DF90BF9002
:1062B000AF900895DC011C96ED91FC911D97E05C78
:1062C000FF4F2191319180819181281B390B2F73D0
:1062D0003070C9010895DC011C96ED91FC911D9769
:1062E000E05CFF4F20813181E054F040DF01AE5B84
:1062F000BF4F8D919C9111972817390719F42FEFF3
:106300003FEF07C08D919C91E80FF91F8081282FE6
:1063100030E0C9010895DC011C96ED91FC911D97B8
:10632000E05CFF4F20813181E054F040DF01AE5B43
:10633000BF4F8D919C9111972817390719F42FEFB2
:106340003FEF10C08D919C911197E80FF91F2081AC
:106350008D919C91119701968F73907011969C93DB
:106360008E9330E0C9010895DC0191968C9191974C
:10637000882339F05496ED91FC915597808186FFE2
:10638000F9CF91961C920895CF93DF93EC01EE859F
:10639000FF85E05CFF4F20813181E054F0402F5FAA
:1063A0003F4F2F733070DF01AE5BBF4F8D919C91DB
:1063B000119728173907D1F3E05CFF4F8081918155
:1063C000E054F040E80FF91F6083EE85FF85E05C44
:1063D000FF4F31832083EE89FF89208181E090E0A7
:1063E0000F8C02C0880F991F0A94E2F7282B208394
:1063F00081E089A3EC89FD8980818064808381E0CC
:1064000090E0DF91CF91089581E008951092BD074B
:106410001092BC0788EE93E0A0E0B0E08093BE0746
:106420009093BF07A093C007B093C10789E995E097
:106430009093BB078093BA0782E397E09093C707D6
:106440008093C60786E797E09093C9078093C807B3
:1064500085EC90E09093CB078093CA0784EC90E0A2
:106460009093CD078093CC0780EC90E09093CF077A
:106470008093CE0781EC90E09093D1078093D00772
:1064800082EC90E09093D3078093D20786EC90E063
:106490009093D5078093D40784E08093D60783E058
:1064A0008093D70787E08093D80785E08093D9074A
:1064B00081E08093DA070895CF93DF930E94062F3F
:1064C0000E945112C5E8D0E30E94661C2097E1F3B8
:1064D0000E948530F9CFCF92DF92EF92FF920F9317
:1064E0001F93CF93DF937C016B018A01C0E0D0E062
:1064F0000FC0D6016D916D01D701ED91FC91019016
:10650000F081E02DC7010995C80FD91F0150104037
:106510000115110571F7CE01DF91CF911F910F91F8
:10652000FF90EF90DF90CF900895DC01ED91FC910A
:106530000190F081E02D09950895EF92FF920F935D
:106540001F938C01DC01ED91FC910190F081E02D15
:106550006DE009957C01D801ED91FC910190F081ED
:10656000E02DC8016AE009959C012E0D3F1DC9016F
:106570001F910F91FF90EF900895CF93DF93EC015F
:106580006115710519F420E030E00FC0DB010D90BA
:106590000020E9F71197A61BB70BE881F98102806B
:1065A000F381E02DAD0109959C01C901DF91CF91E7
:1065B00008954F925F927F928F929F92AF92BF9277
:1065C000CF92DF92EF92FF920F931F93DF93CF93BF
:1065D000CDB7DEB7A1970FB6F894DEBF0FBECDBF23
:1065E0002C01742ECB01223008F42AE019A231E2EA
:1065F000C32ED12CCC0EDD1E822E9924AA24BB24BE
:10660000672D752FA50194010E949A3479018A01A2
:10661000C801B701A50194010E945434472D461BBF
:106620000894C108D1084A3014F4405D01C0495CA7
:10663000F6014083E114F1040105110521F07E2CDF
:106640005F2DC801DDCFC201B6010E94BD32A19607
:106650000FB6F894DEBF0FBECDBFCF91DF911F9173
:106660000F91FF90EF90DF90CF90BF90AF909F90F1
:106670008F907F905F904F900895DC012115310538
:1066800041F4ED91FC910190F081E02D642F09958A
:1066900008950E94D9320895EF92FF920F931F93AD
:1066A0009A01E62EFF2400E010E0B801A7010E9445
:1066B0003D331F910F91FF90EF900895CF92DF929D
:1066C000EF92FF920F931F936C01E62E9A01FF2425
:1066D00000E010E0B801A7010E943D338C01C60123
:1066E0000E949D32080F191FC8011F910F91FF9042
:1066F000EF90DF90CF900895CF92DF92EF92FF92CC
:106700000F931F93CF93DF93EC016A017B01211557
:10671000310541F4E881F9810190F081E02D642F89
:1067200009951FC02A303105D1F477FF17C0E881E1
:10673000F9810190F081E02D6DE209958C014427EB
:106740005527BA014C195D096E097F09CE012AE06F
:106750000E94D9329801280F391F04C02AE00E94F4
:10676000D9329C01C901DF91CF911F910F91FF9008
:10677000EF90DF90CF900895EF92FF920F931F93C9
:106780007B019A010027F7FC0095102FB801A701A3
:106790000E947C331F910F91FF90EF900895CF924C
:1067A000DF92EF92FF920F931F936C017B019A018E
:1067B0000027F7FC0095102FB801A7010E947C3339
:1067C0008C01C6010E949D32080F191FC8011F913C
:1067D0000F91FF90EF90DF90CF9008950E94BD320F
:1067E0000895EF92FF920F931F937C010E94BD3298
:1067F0008C01C7010E949D32080F191FC8011F910B
:106800000F91FF90EF900895CF93DF93EC010E94DA
:10681000952E688779878A879B87E881F98106802A
:10682000F781E02DCE0109959C0197FF15C00E94CC
:10683000952E288539854A855B85621B730B840BF1
:10684000950B2C813D814E815F8162177307840710
:10685000950718F32FEF3FEFC901DF91CF9108950E
:10686000CF92DF92EF92FF920F931F93CF93DF931C
:106870006C018B017A01C0E0D0E009C0C6010E9422
:10688000043497FD07C0F80181938F012196CE153E
:10689000DF05A0F3CE01DF91CF911F910F91FF9003
:1068A000EF90DF90CF900895629FD001739FF00129
:1068B000829FE00DF11D649FE00DF11D929FF00D90
:1068C000839FF00D749FF00D659FF00D9927729FC7
:1068D000B00DE11DF91F639FB00DE11DF91FBD0152
:1068E000CF0111240895AA1BBB1B51E107C0AA1FA9
:1068F000BB1FA617B70710F0A61BB70B881F991F61
:106900005A95A9F780959095BC01CD01089597FB04
:10691000092E07260AD077FD04D0E5DF06D0002037
:106920001AF4709561957F4F0895F6F790958195CB
:106930009F4F0895A1E21A2EAA1BBB1BFD010DC09B
:10694000AA1FBB1FEE1FFF1FA217B307E407F5071F
:1069500020F0A21BB30BE40BF50B661F771F881FFB
:10696000991F1A9469F760957095809590959B0191
:10697000AC01BD01CF01089597FB092E05260ED06D
:1069800057FD04D0D7DF0AD0001C38F4509540954D
:10699000309521953F4F4F4F5F4F0895F6F79095F3
:1069A0008095709561957F4F8F4F9F4F0895EE0FA3
:1069B000FF1F0590F491E02D09942F923F924F9282
:1069C0005F926F927F928F929F92AF92BF92CF927F
:1069D000DF92EF92FF920F931F93CF93DF93CDB788
:1069E000DEB7CA1BDB0B0FB6F894DEBF0FBECDBF00
:1069F00009942A88398848885F846E847D848C84D1
:106A00009B84AA84B984C884DF80EE80FD800C81D9
:106A10001B81AA81B981CE0FD11D0FB6F894DEBFBC
:0C6A20000FBECDBFED010895F894FFCF2C
:106A2C002E003F50313D002650323D0028002900F9
:106A3C002650333D002650343D002650323D310067
:106A4C0047455420002F20002C200001000000544A
:106A5C005556212223C0A80119C0A80101C0A801C4
:106A6C0001C0A80101FFFFFF00501A4F9033C8323C
:106A7C0040003A00204E00001027000002000000E9
:106A8C0000000000000000000000000000000000FA
:106A9C0000000000000000000000000000000000EA
:106AAC0000000000000000000000000000000000DA
:106ABC0000000000000000000000000000000000CA
:106E9C000000000000000000000000000000417233
:106EAC006475696E6F2D3030000A01010001500AC3
:106EBC002C0100000100000000C4316B325A318BF0
:066ECC00316B31B431000E
:00000001FF
